:020000040000FA
:100000000C94E6010C940E020C940E020C94DB1D71
:100010000C94DB1D0C94DB1D0C940E020C940E0250
:100020000C940E020C940E020C940E020C940E0210
:100030000C940E020C940E020C940E020C940E0200
:100040000C94911D0C940E020C945F1D0C94391DA0
:100050000C940E020C940E020C940E020C940E02E0
:100060000C94531E0C940E0207634236B79BD8A71C
:100070001A39685618AEBAAB558C1D3CB7CC5763CD
:10008000BD6DEDFD753EF6177231BF000000803F7B
:1000900008000000BE922449123EABAAAA2ABECD97
:1000A000CCCC4C3E00000080BEABAAAAAA3E000009
:1000B0000000BF000000803F000000000008417801
:1000C000D3BB4387D1133D190E3CC3BD4282AD2B38
:1000D0003E68EC8276BED98FE1A93E4C80EFFFBE30
:1000E00001C4FF7F3F00000000004E414E494E49D1
:1000F0005459494E46CDCCCC3D0AD7233C17B7D1F5
:100100003877CC2B329595E6241FB14F0A0000209A
:10011000410000C84200401C4620BCBE4CCA1B0E19
:100120005AAEC59D7400407A10F35A00A0724E1862
:10013000090010A5D4E80000E87648170000E40B99
:1001400054020000CA9A3B000000E1F5050000805F
:10015000969800000040420F000000A086010000B9
:1001600000102700000000E8030000000064000009
:100170000000000A00000000000100000000002C48
:1001800076D888DC674F0823DFC1DFAE59E1B1B70D
:1001900096E5E3E453C63AE651997696E8E6C284DA
:1001A00026EB898C9B62ED407C6FFCEFBC9C9F40F2
:1001B000F2BAA56FA5F490055A2AF75C936B6CF917
:1001C000676DC11BFCE0E40D47FEF520E6B500D0ED
:1001D000ED902E0300943577050080841E08000002
:1001E000204E0A000000C80C333333330F986E12D0
:1001F000831141EF8D2114893BE65516CFFEE6DBD6
:1002000018D1844B381BF77C1D901DA4BBE424201F
:100210003284725E228100C9F124ECA1E53D2754AD
:100220003D004E6F20445320546865726D6F6D65BC
:10023000746572210020572F6D5E3220555620497B
:100240006E74656E73697479002353656E736F7293
:10025000206572726F722100234E6F20504D207303
:10026000656E736F722100504D28312E302C322E66
:10027000352C3130293D00206C78204C696768743A
:1002800020496E74656E7369747900495220466C1A
:10029000616D65204C6576656C3D00476173206C2F
:1002A0006576656C3D0023496E76616C6964206BF0
:1002B00065792100005EBCE2613FDD83C29C7E2047
:1002C000A3FD1F41009D23BE46DB65F88C11AF32B4
:1002D000CA57E97400000000240027002A002362A6
:1002E0006D70206661696C6564002357656C636F8F
:1002F0006D6520746F20757365204E616E6F204CA4
:100300006F67676572004D533D00235556207A652F
:10031000726F20766F6C74616765203D00503D0000
:1003200042543D004448543D002344757261746951
:100330006F6E3D0054494D45443D0023496E746540
:100340007276616C3D0054494D45493D0053484F1C
:1003500057533D004C6F67676572204E616D653A7B
:1003600020004C4F474745520056455253494F4E87
:10037000005245424F4F54000000000800020100A7
:10038000000304070000000000000000000000005F
:1003900023002600290000000000250028002B0073
:1003A000040404040404040402020202020203031B
:1003B0000303030301020408102040800102040823
:1003C0001020010204081020721FD92711241FBE1B
:1003D000CFEFD8E0DEBFCDBF12E0A0E0B1E0E0E5B6
:1003E000F9E602C005900D92A631B107D9F724E0D5
:1003F000A6E1B2E001C01D92A93AB207E1F711E00F
:10040000C5EED1E004C02197FE010E947E32C43EB9
:10041000D107C9F70E94D4200C949B340C9400009F
:10042000089508950895AF92BF92CF92DF92EF9210
:10043000FF920F931F93CF93DF936C017B018B018E
:10044000040F151FEB015E01AE18BF08C017D107DE
:1004500059F06991D601ED91FC910190F081E02D68
:10046000C6010995892B79F7C501DF91CF911F91BD
:100470000F91FF90EF90DF90CF90BF90AF900895D5
:10048000CF93DF93FC01448155816081718189E2C2
:1004900093E00E941302EC0142E050E069E571E054
:1004A00089E293E00E9413028C0F9D1FDF91CF9190
:1004B0000895FC01538D448D252F30E0842F90E06A
:1004C000821B930B541710F0CF960895019708954F
:1004D000FC01918D828D981761F0A28DAE0FBF2F18
:1004E000B11D5D968C91928D9F5F9F73928F90E06E
:1004F00008958FEF9FEF0895FC01918D828D9817DD
:1005000031F0828DE80FF11D858D90E008958FEF19
:100510009FEF0895FC01918D228D892F90E0805CE2
:100520009F4F821B91098F739927089589E293E069
:100530000E948A0221E0892B09F420E0822F08958D
:1005400080E090E0892B29F00E94960281110C94A2
:1005500000000895FC01A48DA80FB92FB11DA35A66
:10056000BF4F2C91848D90E001968F739927848FD3
:10057000A689B7892C93A089B1898C9183708064F6
:100580008C93938D848D981306C00288F389E02D97
:1005900080818F7D80830895EF92FF920F931F9348
:1005A000CF93DF93EC0181E0888F9B8D8C8D981326
:1005B0001AC0E889F989808185FF15C09FB7F89432
:1005C000EE89FF896083E889F9898081837080647E
:1005D00080839FBF81E090E0DF91CF911F910F91C9
:1005E000FF90EF900895F62E0B8D10E00F5F1F4FD8
:1005F0000F731127E02E8C8D8E110CC00FB607FCE7
:10060000FACFE889F989808185FFF5CFCE010E9474
:10061000AA02F1CFEB8DEC0FFD2FF11DE35AFF4F36
:10062000F0829FB7F8940B8FEA89FB898081806202
:10063000CFCFCF93DF93EC01888D8823B9F0AA89BF
:10064000BB89E889F9898C9185FD03C0808186FD8D
:100650000DC00FB607FCF7CF8C9185FFF2CF8081DC
:1006600085FFEDCFCE010E94AA02E9CFDF91CF91A5
:100670000895833081F028F4813099F08230A9F018
:1006800008958730A9F08830C9F08430B1F48091A2
:1006900080008F7D03C0809180008F7780938000E1
:1006A000089584B58F7784BD089584B58F7DFBCF81
:1006B0008091B0008F778093B00008958091B00052
:1006C0008F7DF9CFCF93DF93E7E8F3E08491E3ECFC
:1006D000F3E0D491EFEAF3E0C491CC23A1F08111CF
:1006E0000E943903EC2FF0E0EE0FFF1FE457FC4FA0
:1006F000A591B491EC91ED2381E090E009F480E0C4
:10070000DF91CF91089580E090E0FACF1F93CF93CF
:10071000DF93282F30E0F901E858FC4F8491F9016C
:10072000EC54FC4FD491F901E056FC4FC491CC231A
:10073000A9F0162F81110E943903EC2FF0E0EE0F83
:10074000FF1FEA56FC4FA591B4918FB7F894EC9136
:10075000111108C0D095DE23DC938FBFDF91CF91BC
:100760001F910895DE2BF8CFCF93DF9390E0FC012B
:10077000EC54FC4F249180569C4FFC0184918823BB
:10078000D1F090E0880F991FFC01EC52FD4FA5912C
:10079000B491FC01EA56FC4FC591D49161110EC091
:1007A0009FB7F8948C91E22FE0958E238C9328814B
:1007B000E223E8839FBFDF91CF9108958FB7F8942C
:1007C000EC91E22BEC938FBFF6CF8E3008F08E5079
:1007D0002091000190E4299F900111248770822BC1
:1007E00080937C0080917A00806480937A0080916D
:1007F0007A0086FDFCCF8091780090917900089571
:100800003FB7F89480919F029091A002A091A1021D
:10081000B091A20226B5A89B05C02F3F19F0019602
:10082000A11DB11D3FBFBA2FA92F982F8827BC014A
:10083000CD01620F711D811D911D42E0660F771F72
:10084000881F991F4A95D1F708958F929F92AF9272
:10085000BF92CF92DF92EF92FF926B017C010E94D8
:1008600000044B015C01C114D104E104F104B9F0AE
:100870000E940004681979098A099B09683E73403F
:100880008105910580F321E0C21AD108E108F10841
:1008900088EE880E83E0981EA11CB11CE4CFFF9067
:1008A000EF90DF90CF90BF90AF909F908F90089582
:1008B0008F929F92AF92BF92EF92FF921F93CF932E
:1008C000DF93C82F10929D0410929E0410929F04F3
:1008D0001092A0041092A10461E08FE00E94B40382
:1008E00060E08FE00E9486036C2F70E090E080E073
:1008F0000E94250460E08FE00E94B4038BE990E041
:100900000197F1F7C0E9D1E00E946203892B71F4ED
:100910002197D1F78EEF9FEFDF91CF911F91FF903D
:10092000EF90BF90AF909F908F900895C0E9D1E075
:100930000E946203019719F42197D1F7EBCFD8E217
:10094000C0E810E090E9E92EFF24F3940E946203CE
:10095000892B29F481E0E81AF108C1F7DBCF0E9466
:1009600000044B015C0180E9E82EFF24F3940E940F
:100970006203019729F481E0E81AF108C1F7CACFB0
:100980000E940004681979098A099B096932710576
:100990008105910538F0E12FF0E0EB56FB4F8085A3
:1009A0008C2B8087C69511F41F5FC0E8D15051F69B
:1009B00090E080E0B1CF8F929F92AF92BF92CF92A2
:1009C000DF92EF92FF920F931F93CF93DF938AE012
:1009D000A82EB12CD0E0C0E0EE24EA9493E0F92EEA
:1009E00088248A9423E0922ED12CC12C10E000E0C0
:1009F0008FE00E94E5030817190790F1C816D90681
:100A000008F46C018815990568F18E159F0508F4A6
:100A10007C01C80FD91F65E070E080E090E00E9483
:100A2000250481E0A81AB10819F70C0D1D1DCE018F
:100A3000801B910B8E199F098819990966E070E057
:100A40000E940A31CB01DF91CF911F910F91FF904E
:100A5000EF90DF90CF90BF90AF909F908F900895D0
:100A60008C01D0CF4C01D5CF2FB7F89460919B0269
:100A700070919C0280919D0290919E022FBF0895DB
:100A8000DC0180E0615090F09D919827E92FEF7094
:100A9000F0E0EC54FD4F2491E92FE295EF70F0E087
:100AA000EC53FD4FE491822F8E27ECCF0895DC01AB
:100AB0002C911196ED91FC91F8948181822B818388
:100AC0009281322F30959323928387E090E00197B3
:100AD000F1F781818323818383E290E00197F1F72D
:100AE00090817894EFECF0E03197F1F7922381E078
:100AF00009F480E00895FC0190810180F281E02DED
:100B0000292F209560FF14C0F8948281822382836C
:100B10008181892B8183A3E2B0E01197F1F7828173
:100B2000982B9283789487ED90E00197F1F70895E0
:100B3000F8948281822382838181892B8183AFEF24
:100B4000B0E01197F1F78281982B928378948FE02F
:100B500090E0EBCFDF92EF92FF920F931F93CF9332
:100B6000DF93EC01D62EE42E08E010E0FF24F3948E
:100B700061E08D2D8F2109F460E0CE010E947B059C
:100B8000FF0C01501109A1F7E11010C0F894E981A0
:100B9000FA8191818881809589238183E981FA8115
:100BA000928188818095892382837894DF91CF9187
:100BB0001F910F91FF90EF90DF900895EF92FF92B9
:100BC0000F931F93CF93DF938C017B0140E065E58A
:100BD0000E94AA05E70188E0E80EF11C699140E057
:100BE000C8010E94AA05CE15DF05C1F7DF91CF919C
:100BF0001F910F91FF90EF900895FC01908101806B
:100C0000F281E02DF8948181292F20958223818320
:100C100078943DE743E050E0315029F1DA01119733
:100C2000F1F780818923C1F3F89482818223828342
:100C30008181892B81837894ABE7B7E01197F1F735
:100C4000F894818182238183A3E1B1E01197F1F7C8
:100C50008081982381E009F080E07894E3E6F6E073
:100C60003197F1F7089580E008956F927F928F9207
:100C70009F92AF92BF92CF92DF92EF92FF920F932B
:100C80001F93CF93DF93EC017B018A018E819F81BB
:100C90000E94FD05811102C090E037C0B7018E812E
:100CA0009F810E94DE0540E06EEB8E819F810E9455
:100CB000AA057801680189E0C80ED11CAE80BF800A
:100CC00088E0882E912C712C66246394C5010E94C3
:100CD000570581117628660CE1E08E1A9108B1F76C
:100CE000F70171927F01EC15FD0541F78E819F811F
:100CF0000E94FD05813081F668E0C8010E94400530
:100D000091E0F80120852813C7CF892FDF91CF917B
:100D10001F910F91FF90EF90DF90CF90BF90AF9019
:100D20009F908F907F906F900895CF93DF93CDB772
:100D3000DEB729970FB6F894DEBF0FBECDBFAE0168
:100D40004F5F5F4F0E943506882331F08D818F33CE
:100D5000A9F020F48F31A1F080E007C08F3521F099
:100D60008F37D1F78CE001C08BE029960FB6F8944D
:100D7000DEBF0FBECDBFDF91CF9108958AE0F5CFE2
:100D800089E0F3CF2091B5023091B60228173907D8
:100D900071F49091B3028091B402981741F0E09100
:100DA000B302F0E0E65AFD4F808190E008958FEFA6
:100DB0009FEF08950895EF92FF920F931F93CF93A3
:100DC000DF93DC015C96ED90FC905D97E114F104FB
:100DD00079F481E090E013969C938E93129790E0C3
:100DE00080E0DF91CF911F910F91FF90EF900895D8
:100DF0005196ED91FC91529750968C915097982F67
:100E000090950FB75E962C915E97122F127021FD70
:100E10006095F8942081112319F1282B2083E70194
:100E20002197F1F728E0462F50E0308160FF1AC08B
:100E3000382B3083E7012197F1F7BA017595679553
:100E4000215089F7112381F08081892380830FBF8E
:100E50005C968D919C910197F1F781E090E0C1CF74
:100E60002923DCCF3923E5CF9081892BEFCF209147
:100E7000B5023091B6022817390771F48091B40297
:100E80002091B30290E0805C9F4F821B910960E447
:100E900070E00E941E31089590E080E00895209156
:100EA000B5023091B60228173907B9F49091B30210
:100EB0008091B402981789F0E091B302F0E0E65A0D
:100EC000FD4F80812091B30230E02F5F3F4F2F73A1
:100ED00033272093B30290E008958FEF9FEF08959A
:100EE0000F931F930E94340560937E0470937F04D8
:100EF000809380049093810486E794E00E944F07DA
:100F000097FF1DC00E94340500917E0410917F045C
:100F10002091800430918104601B710B820B930B34
:100F200000917A0410917B0420917C0430917D041F
:100F30006017710782079307F8F28FEF9FEF1F91F9
:100F40000F910895E091B502F091B602E817F90704
:100F500069F4A389B4899C918589809589238C93B0
:100F60001092B6021092B50281E0089580E00895D3
:100F7000109291041092900410928F0410928E049B
:100F800010928D0410928C048DE991E0909393045B
:100F90008093920490918204963108F046C02DEB24
:100FA00030E030938D0420938C042BE931E03093B2
:100FB0008F0420938E042CE231E03093910420932F
:100FC00090042091680084E0983048F031E09E3031
:100FD00008F430E081E001C0880F3A95EAF7822BEF
:100FE000809368002DE630E0983050F02BE630E03A
:100FF0009E3030F02CE630E0963110F030E020E00A
:1010000030938A0420938904292F30E09830C0F56A
:1010100081E001C0880F9A95EAF780938B04809154
:101020009204909193040197F1F78091900490912C
:101030009104892B21F18091B5029091B60224E0B0
:1010400086379207E1F0009711F00E94A207809185
:1010500094048E7F809394041092B4021092B30291
:1010600086E794E09093B6028093B502E0918904FC
:10107000F0918A04808190918B04892B808308955C
:101080009E3040F42850310981E001C0880F2A9534
:10109000EAF7C3CF2E503109F7CF20913702260F40
:1010A0003327331F21323105ECF42091FF02FC017C
:1010B00090E080E0243069F082E00895A09137024A
:1010C0002191AC01495E5D4FA40FB52FB11D2C934A
:1010D0000196861798F380913702680F6093370264
:1010E00080E0089581E008951092FF0281E08093EE
:1010F000FE021092D90261E082E10E94860361E063
:1011000083E10E948603E9EBF0E080818E7F80839B
:1011100080818D7F808388E48093B80085E480930C
:10112000BC0008951092B8021092B7021092060304
:10113000109228030E94740880E192E09093B2021A
:101140008093B10281E192E09093B0028093AF026C
:101150000895CF93DF9391E0909316028823B9F01E
:10116000C091B800D091BA008091BC008A7B809376
:10117000BC0060E082E10E94860360E083E10E949F
:1011800086030E947408D093BA00C093B800DF9120
:10119000CF910895CF92DF92EF92FF920F931F931A
:1011A000CF93DF93D091280381E0D13208F09CC027
:1011B000C09127030E9400046B017C018091FF0213
:1011C00081116CC082E08093FF0281E08093FE0277
:1011D0008FEF8093FD021092FC02D093FB02A7E0F8
:1011E000B3E0EBEDF2E080E0D8138DC01092DA02AC
:1011F0008091DA02CC0FC82BC093DA028091D90219
:10120000813009F084C01092D9020E9400046B0161
:101210007C018091DA028093BB0080910103909160
:101220000203A0910303B0910403892B8A2B8B2B1B
:10123000A1F00E940004009101031091020320918B
:101240000303309104036C197D098E099F09061769
:1012500017072807390708F442C08091BC0083FDB6
:10126000D8CF85EC8093BC000E9400046B017C0108
:101270008091FF02823009F44CC08091FD028F3FC3
:1012800009F469C08091FD02803209F466C0809142
:10129000FD02803309F463C084E026C0809101031D
:1012A00090910203A0910303B0910403892B8A2B30
:1012B0008B2B09F483CF0E9400040091010310914D
:1012C000020320910303309104036C197D098E09F8
:1012D0009F09061717072807390708F06FCF809175
:1012E00000030E94A90885E01092060310922803CB
:1012F00010920503DF91CF911F910F91FF90EF9016
:10130000DF90CF9008959D9191938F5F6DCF85EE83
:10131000A9CF8091010390910203A0910303B091A2
:101320000403892B8A2B8B2B09F4A2CF0E94000483
:1013300000910103109102032091030330910403F3
:101340006C197D098E099F090617170728073907A9
:1013500008F08ECFC4CF80E0C7CF82E0C5CF83E056
:10136000C3CFCF92DF92EF92FF920F931F93CF9351
:10137000DF93D82FC62F613208F098C00E94000476
:101380006B017C018091FF0281116BC081E0809331
:10139000FF028093FE029FEF9093FD021092FC02E9
:1013A0009C0F9093FB028093DA028091DA02DD0FAA
:1013B000D82BD093DA028091D902813009F078C01D
:1013C0001092D9020E9400046B017C018091DA0224
:1013D0008093BB008091010390910203A0910303CD
:1013E000B0910403892B8A2B8B2BA1F00E9400045F
:1013F0000091010310910203209103033091040333
:101400006C197D098E099F090617170728073907E8
:1014100008F448C08091BC0083FDD8CF85EC809350
:10142000BC000E9400046B017C018091FF028130AE
:1014300009F440C08091FC028C1710F4C091FC02AA
:10144000EBEDF2E0A9EBB2E080E08C1355C08C2FFD
:10145000DF91CF911F910F91FF90EF90DF90CF9090
:1014600008958091010390910203A0910303B0912C
:101470000403892B8A2B8B2B09F484CF0E94000450
:1014800000910103109102032091030330910403A2
:101490006C197D098E099F09061717072807390758
:1014A00008F070CF809100030E94A908C0E0CFCF60
:1014B00085EEB5CF8091010390910203A0910303C3
:1014C000B0910403892B8A2B8B2B09F4AECF0E9499
:1014D0000004009101031091020320910303309155
:1014E00004036C197D098E099F0906171707280741
:1014F000390708F09ACFD6CF91919D938F5FA5CFF2
:10150000E091B8028091B702E81730F4F0E0E754B8
:10151000FD4F808190E008958FEF9FEF08959091A7
:10152000B8028091B7022FEF3FEF981748F4E92FE8
:10153000F0E0E754FD4F208130E09F5F9093B802C8
:10154000C90108958091B7029091B802891B990B47
:101550000895CF92DF92EF92FF920F931F93CF9354
:10156000DF937C01CB018A0120910503222389F0BE
:10157000EB016B01C40ED51ECC15DD0569F0699138
:10158000D701ED91FC910190F081E02DC701099503
:10159000F3CF642F0E944D08C801DF91CF911F91B6
:1015A0000F91FF90EF90DF90CF900895CF93DF934E
:1015B0001F92CDB7DEB76983209105032223F9F08E
:1015C00020912803203258F021E030E0FC013383E1
:1015D000228390E080E00F90DF91CF910895809179
:1015E0000603E82FF0E0E95FFC4F998190838F5F5D
:1015F000809306038093280381E090E0ECCF61E0C4
:10160000CE0101960E944D08F7CF90E080E008954A
:1016100086E794E00E94A2070C94B8072F923F92AD
:101620004F925F926F927F928F929F92AF92BF92F2
:10163000CF92DF92EF92FF920F931F93CF93DF939E
:10164000CDB7DEB72D970FB6F894DEBF0FBECDBF76
:101650001C010E94080B64E670E080E090E00E94AC
:1016600025046AE070E080E090E00E942504C1015A
:10167000880F991F9D878C87D12CC12CF12CE12CD0
:10168000412C512C320149E050E06AE171E086E7DB
:1016900094E00E94130265E070E080E090E00E9418
:1016A000250410E000E0812C912C540186E794E0A1
:1016B0000E943707892B39F4F4E08F169104A104B6
:1016C000B1040CF05FC0023011050CF05BC086E77E
:1016D00094E00E943707892B99F086E794E00E94F6
:1016E0004F07E1E0F0E0EC0FFD1FE00FF11F8083FA
:1016F0006AE070E080E090E00E9425040F5F1F4FD9
:1017000065E070E080E090E00E9425040230110561
:1017100009F070C089818F3F09F06CC08A818638DA
:1017200009F068C0FE013396FB87EA8786E794E0FC
:101730000E943707892B39F4F4E08F169104A10435
:10174000B1040CF050C00930110509F059C08B816B
:1017500090E0982F88272C81820F911D092E000C74
:10176000AA0BBB0B480E591E6A1E7B1E40C0EC859F
:10177000FD85EC15FD0509F086CFE114F10441F477
:10178000710106C08FEFC81AD80AE214F3047CF383
:10179000C301B2010E94512C4B015C01B701FF0C47
:1017A000880B990B0E94512C9B01AC01C501B4011F
:1017B0000E946F2E2D960FB6F894DEBF0FBECDBFE0
:1017C000DF91CF911F910F91FF90EF90DF90CF901D
:1017D000BF90AF909F908F907F906F905F904F9051
:1017E0003F902F900895043011050CF0B0CFFFEF1B
:1017F000EF1AFF0A8FEF881A980AA80AB80A56CF7C
:1018000086E794E00E944F07EA85FB858193FB877A
:10181000EA870F5F1F4F8ACF8F929F92AF92BF923E
:10182000CF92DF92EF92FF92CF93DF93C8E4D4E0A0
:10183000988121E0209305039093270310920603DB
:1018400010922803682F86EC93E00E94D60A0E942B
:10185000CA0863E088810E94B1091092B80280939F
:10186000B70286EC93E00E948F0A092E000CAA0BA7
:10187000BB0B8824982EA92EBA2E86EC93E00E94EA
:101880008F0A092E000CAA0BBB0B6C017D01C82826
:10189000D928EA28FB28FE2CED2CDC2CCC2486EC65
:1018A00093E00E948F0ABC01990F880B990B6C2959
:1018B0007D298E299F29DF91CF91FF90EF90DF90B6
:1018C000CF90BF90AF909F908F9008958F929F92EE
:1018D000AF92BF92CF92DF92EF92FF920F931F933E
:1018E000209151042F3F19F48AEF0E940C0C0091B3
:1018F00055041091560430E020E0C72ED82EE92E72
:10190000FF24E7FCFA94C01AD10AE20AF30A57E06E
:1019100095958795779567955A95D1F7000F111F83
:10192000221F331F4B015C01801A910AA20AB30ADD
:10193000A5019401A0915704B09158040E94922DE2
:101940004B015C01FBE0B594A79497948794FA95BA
:10195000D1F7A7019601C701B6010E94FA309B0199
:10196000AC01ACE05595479537952795AA95D1F7E9
:10197000A0915904B0915A040E94922D9B01AC0190
:10198000BEE05595479537952795BA95D1F7280D1F
:10199000391D4A1D5B1D20934D0430934E04409326
:1019A0004F0450935004A5E0B0E00E94872D60588A
:1019B0007F4F8F4F9F4F672F782F892F992787FD54
:1019C0009A950E94512C20E030E048EC52E40E94AD
:1019D0006F2E1F910F91FF90EF90DF90CF90BF90EF
:1019E000AF909F908F9008952F923F924F925F9269
:1019F0006F927F928F929F92AF92BF92CF92DF921F
:101A0000EF92FF920F931F93CF93DF93CDB7DEB783
:101A10006B970FB6F894DEBF0FBECDBF0E94660C69
:101A2000809151048F3F39F487EF0E940C0C6E8B2C
:101A30007F8B888F998F80914D0490914E04A09157
:101A40004F04B09150046C017D01FF0CCC08DC2CDC
:101A500076019C01AD016C2D7C2D8C2D9C2D345F6D
:101A600041405109610971098109910929873A8722
:101A70004B87652E762E872E982E9B8F5901C42E6C
:101A8000D52EE62EF72E082F192F0E943231322E36
:101A9000232E488B598B6A8B7B8B8C8B9D8B309143
:101AA0005E0420915D04932F990F990B492F592FB4
:101AB000692F792F892F0E9432310CE00E942A323F
:101AC00029833C874A8F5D876E877F87582E492EF2
:101AD0003091600420915F04932F990F990BA32CF0
:101AE000B22CC888D988EA88FB880C891D89492FBF
:101AF000592F692F792F892F0E94323108E00E94D7
:101B00004332A980BC84CA8CDD84EE84FF84052D19
:101B1000142D0E94603270588F4F9F4FE0915B04EC
:101B2000F0915C045F01D12CC12CE12CF12C8701D8
:101B3000E983BA82CB82DC82ED82FE820F83188732
:101B4000C12CD12CE12CF12C00E010E00E943231AC
:101B500001E20E9443322A8F532E49835C876D87AE
:101B60007E878F87492EA0E00E94723209F436C129
:101B70003091660420916504932F990F990BA32C43
:101B8000B22CC888D988EA88FB880C891D89492F1E
:101B9000592F692F792F892F0E9432311901488BD3
:101BA000598B6A8B7B8B8C8B9D8B3091640420913D
:101BB0006304932F990F990BA984BA84CB84D62CF4
:101BC000E72CF82C092D1B8D492F592F692F792FC0
:101BD000892F0E94323101E10E942A325101C888C6
:101BE000D988EA88FB880C891D890E9460325901D6
:101BF0006A017B01382E192F4E895F89688D798D96
:101C000084E075956795579547958A95D1F780E05B
:101C100090E0A0E1B0E0841B950BA60BB70B3C0154
:101C20004D01990C6608762C43019C01AD01662D8F
:101C3000762D862D962D0FE10E942A32722E832E4C
:101C4000942E5987B62FA72FF82FE92F30916204D1
:101C500020916104932F990F990B492F592F692FC8
:101C6000792F892F03E20E942A32032D0E946032CD
:101C700059016A017B018C01272D382D492D598589
:101C80006B2F7A2F8F2F9E2F0E946932E5E3AE2EA5
:101C9000FCE0BF2EC12CD12CE12CF12C00E010E097
:101CA0000E943231AA8CB52CC980DC84ED84FE847C
:101CB0000F85142D0E948C312F873E8749875A87C4
:101CC0006B8779838C879D870DE00E944332922E2B
:101CD000832E742E652E562E472E382E292E3091A7
:101CE0006C0420916B04932F990F990BA92CB82C9D
:101CF000C72CD62CE52CF42C032D122D492F592F4F
:101D0000692F792F892F0E9432310E94323109E1E7
:101D10000E944332AF84BE84C984DA84EB84F980A4
:101D20000C851D850E94603219012A013B014C017E
:101D300030916A0420916904932F990F990B492FD0
:101D4000592F692F792F892F0E94323103E10E9488
:101D5000433259016A017B018C019101A201B30157
:101D6000C4010E94603208E00E94433259016A01B6
:101D70007B01E82F192F3091680420916704932F7D
:101D8000990F990B492F592F692F792F892F04E02B
:101D90000E942A320E2F0E9460320E94172F20E0EC
:101DA00030E040E85BE30E94B02C6B960FB6F894ED
:101DB000DEBF0FBECDBFDF91CF911F910F91FF907E
:101DC000EF90DF90CF90BF90AF909F908F907F90DB
:101DD0006F905F904F903F902F90089560E070E07B
:101DE000CB01E3CFBF92CF92DF92EF92FF920F939E
:101DF0001F93CF93DF93EC01B62EC72E8D858111F3
:101E000005C0CE010E94FD0581110EC01B861D86F6
:101E10001C8680E0DF91CF911F910F91FF90EF9092
:101E2000DF90CF90BF90089540E060EFCE010E9418
:101E3000AA0501E0E12CD12C11E0CE010E9457054A
:101E4000F82ECE010E94570591E0F91218C081309A
:101E500099F51134D8F2DB86D11002C081E08D876C
:101E60008B81882399F22396EB2DFC2DCF010896C8
:101E700029912193E817F907D9F781E0CBCFEE2D0F
:101E8000F0E0F8120FC08B851817A0F4DE01AE0F3A
:101E9000BF1F13968C91802379F4F12C193008F42C
:101EA0001C87D12EEC0FFD1F8381902F90958923E5
:101EB00083830AC08113F1CFFE01EE0DF11D8381F2
:101EC000802B8383FF24F3946F2DCE010E947B052A
:101ED0001F5F000F11F4E39401E087E08E1508F016
:101EE000ACCFB7CFDF92EF92FF920F931F93CF93B8
:101EF000DF937C018B01D42EDC011696ED91FC91D1
:101F0000138615861486128611861086178216820D
:101F1000158214821382C0E0B801F701868197818F
:101F20000E94F20ED82F882329F0DC1629F0CF5F0B
:101F3000DC1690F7D0E009C067E0C8010E944005B8
:101F4000D80117969C918913F2CF8D2FDF91CF91F5
:101F50001F910F91FF90EF90DF900895CF93909194
:101F600051049F3F41F5682F8091480491E0909380
:101F7000050380932703109206031092280386EC32
:101F800093E00E94D60A0E94CA0862E08091480449
:101F90000E94B1091092B8028093B70286EC93E0D8
:101FA0000E948F0AC82F86EC93E00E948F0A20E0DF
:101FB0003C2F282B392B922F832FCF910895AF924E
:101FC000BF92DF92EF92FF920F931F93CF93DF9315
:101FD0005C0102ED13E0D0E0C0E0F801D1908F0188
:101FE0007501EC0EFD1EC7010E94712DD81621F05F
:101FF0006D2DC7010E94792D2196CC34D10569F74A
:1020000082ED93E0DF91CF911F910F91FF90EF90C0
:10201000DF90BF90AF90089585ED8093BC008091D4
:10202000010390910203A0910303B091040307966A
:10203000A11DB11D23E0B695A795979587952A9583
:10204000D1F72091BC0024FD03C01092FF02089537
:1020500040910103509102036091030370910403C6
:10206000452B462B472B69F30097A105B10541F09D
:1020700025E32A95F1F700000197A109B109E1CF05
:10208000809100030C94A908FC0180819181009744
:1020900011F00C94212860E070E0CB010895FB0161
:1020A00044815581FC01248135812417350778F05E
:1020B00080819181009759F0FB01608171816115E8
:1020C000710529F00E947E3421E0892B09F020E07F
:1020D000822F08950F931F93CF93DF938C01EB0111
:1020E000FC01808191810097E1F06881798161151F
:1020F0007105A9F0428153812C813D81421753071C
:1021000070F00E9477348C819D81F80195838483DF
:102110001D821C82DF91CF911F910F9108950E9423
:10212000203388819981F801918380838A819B8102
:10213000938382838C819D81958384831982188205
:102140001B821A82E5CFCF93DF93EC0188819981BE
:10215000009711F00E942033198218821D821C8280
:102160001B821A82DF91CF910895FC0180819181B9
:10217000009711F00C94203308950F931F93CF9381
:10218000DF93EC0188819981009759F02A813B8186
:102190002617370730F081E0DF91CF911F910F9123
:1021A00008958B016F5F7F4F0E94A933009759F00C
:1021B000998388831B830A832C813D81232B59F7C4
:1021C000FC011082E8CF80E0E7CFEF92FF920F93FF
:1021D0001F93CF93DF936115710541F480E0DF9188
:1021E000CF911F910F91FF90EF90089541155105E8
:1021F000B1F07B01EC010C811D81040F151FB801AA
:102200000E94BD10882351F3288139818C819D81E2
:10221000B701820F931F0E9477341D830C8381E0E6
:10222000DECFFC01448155816081718182E494E0BC
:102230000C94E510CF93DF93EC01FB01019000209B
:10224000E9F73197AF01461B570B0E94E51081114A
:1022500003C0CE010E94A310CE01DF91CF9108955B
:10226000CF93DF93EC01FB01448155816081718143
:102270000E94E510811103C0CE010E94A310CE017F
:10228000DF91CF910895FB0101900020E9F731978C
:10229000AF01461B570B0C94E510EF92FF920F9382
:1022A0001F93CF93DF93EC018B01CB010E944F284A
:1022B0007C01BC01CE010E94BD1081110BC0CE017A
:1022C0000E94A310CE01DF91CF911F910F91FF903B
:1022D000EF900895FD82EC82B801888199810E9477
:1022E0004828F0CFFC0111821082138212821582DD
:1022F00014820C944D11EF92FF920F931F93CF9382
:10230000DF93EC017B018A01BA010E94BD108111AB
:102310000BC0CE010E94A310CE01DF91CF911F917F
:102320000F91FF90EF9008951D830C83B701888172
:1023300099810E947734F0CFFB0101900020E9F7EA
:102340003197AF01461B570B0C947B110F931F93D2
:10235000CF93DF93CDB7DEB762970FB6F894DEBFA9
:102360000FBECDBF8C01CB01F80111821082138208
:102370001282158214824AE0BE016F5F7F4F0E9475
:102380005828BE016F5F7F4FC8010E949C11629662
:102390000FB6F894DEBF0FBECDBFDF91CF911F9176
:1023A0000F910895CF93DF93EC01FB0186179707F8
:1023B00049F0608171816115710541F04481558159
:1023C0000E947B11CE01DF91CF9108950E94A3104E
:1023D000F9CFFC01118210821382128215821482BD
:1023E0000C94D211FC011182108213821282158288
:1023F0001482FB0101900020E9F73197AF01461BE1
:10240000570B0C947B11AF92BF92CF92DF92EF9259
:10241000FF920F931F93CF93DF936C015B017A01BF
:1024200089012417350720F48F2D7901042F182FE7
:102430006BE571E0C6010E94F211D5011496CD91B1
:10244000DC91EC16FD06E0F40C171D0708F4E8011A
:10245000D501ED91FC911197EC0FFD1F10811082B9
:102460006D917C916E0D7F1DC60161157105A1F006
:102470000E949C11F50180819181C80FD91F18839A
:10248000C601DF91CF911F910F91FF90EF90DF90E8
:10249000CF90BF90AF9008950E94A310EBCF0F9301
:1024A0001F93CF93DF93CDB7DEB72C970FB6F89479
:1024B000DEBF0FBECDBFFC0124813581121613068D
:1024C00064F48C01253131059CF40E9440026FE0D8
:1024D00070E080E090E00E9425042C960FB6F894FE
:1024E000DEBF0FBECDBFDF91CF911F910F91089539
:1024F0002FE030E050E040E0BC01CE0107960E94A2
:1025000003124B855C856F81788589E293E00E9498
:10251000130269E170E080E090E00E942504F80178
:10252000248135814FE050E0B801CE0101960E9430
:102530000312BE016F5F7F4FCE0107960E946A10A3
:10254000CE0101960E94B510CE0107960E9440026E
:102550006FE070E080E090E00E9425046BE571E0A0
:10256000CE0107960E949C11CE0107960E94B510DD
:10257000B4CFEF92FF920F931F93CF93DF93CDB71A
:10258000DEB7A1970FB6F894DEBF0FBECDBF7C01BA
:10259000CB01BA01F70111821082138212821582D7
:1025A000148242E0420F8E010F5F1F4F0E94FF27EF
:1025B000009789F0BC01C7010E949C11A1960FB63B
:1025C000F894DEBF0FBECDBFDF91CF911F910F9169
:1025D000FF90EF900895C7010E94A310EFCF8F9254
:1025E0009F92AF92BF92EF92FF920F931F93CF9360
:1025F000DF93CDB7DEB72C970FB6F894DEBF0FBED2
:10260000CDBF64E670E080E090E00E9425048091F8
:102610000401909105010B9731F58091A204882364
:1026200009F0F89482E10E9458048C018091A20480
:10263000882309F078940115110509F4BAC080E0E7
:1026400090ECA9E7B4EC8093950490939604A09342
:102650009704B09398048093990490939A04A0935C
:102660009B04B0939C0480910401909105014697CE
:1026700031F58091A204882309F0F89481E00E944A
:1026800058048C018091A204882309F078940115E4
:10269000110509F4EFC080E090ECA9E7B4EC809359
:1026A000950490939604A0939704B0939804809314
:1026B000990490939A04A0939B04B0939C0464E6BD
:1026C00070E080E090E00E942504012B09F060C0DA
:1026D0004091990450919A0460919B0470919C04DC
:1026E00021E0CE0107960E94B9126CE571E0CE019F
:1026F00001960E94F211BE01695F7F4FCE010196E3
:102700000E9430116FE571E00E941A11BC0182E451
:1027100094E00E94D211CE0101960E94B510409122
:10272000950450919604609197047091980421E06B
:10273000CE0101960E94B912BE016F5F7F4FCE019C
:1027400007960E946A10CE0101960E94B51063E6BA
:1027500071E0CE0101960E94F211BE01695F7F4FC8
:10276000CE0101960E94301166E671E00E941A11B6
:102770000E941111CE0101960E94B51064E670E02E
:1027800080E090E00E942504CE0107960E94B510DB
:102790002C960FB6F894DEBF0FBECDBFDF91CF9160
:1027A0001F910F91FF90EF90BF90AF909F908F90EF
:1027B000089510919D04E0909E046E2D70E090E0CD
:1027C00080E00E94512C2DEC3CEC4CEC5DE30E942F
:1027D000B02C4B015C01612F70E090E080E00E9422
:1027E000512C9B01AC01C501B4010E94032E6093E2
:1027F00095047093960480939704909398040091A5
:102800009F04F090A004602F6F7770E090E080E06C
:102810000E94512C4B015C016F2D70E090E080E034
:102820000E94512C2DEC3CEC4CEC5DE30E94B02C52
:102830009B01AC01C501B4010E94032E07FD18C025
:102840006093990470939A0480939B0490939C04E2
:102850001E0D100F1F0D81E090E02091A1041213B6
:1028600002C090E080E000271127081B190BFBCE67
:102870009058E6CF10919E0400919D0460919D04B4
:1028800070919E0476276727762790E080E00E946B
:102890004F2C2DEC3CEC4CEC5DE30E94B02C609393
:1028A0009504709396048093970490939804E09015
:1028B000A004F0909F046F2D6F77762F6E2D90E01F
:1028C00080E00E944F2C2DEC3CEC4CEC5DE30E9430
:1028D000B02CF7FC18C06093990470939A0480930D
:1028E0009B0490939C04100F1E0D1F0D81E090E03F
:1028F0002091A104121302C090E080E0002711276C
:10290000081B190BDCCE9058E6CF4F925F926F9266
:102910007F928F929F92AF92BF92CF92DF92EF926F
:10292000FF92CF93DF93CDB7DEB72C970FB6F89415
:10293000DEBF0FBECDBF0E94F40C2B013C010E94F4
:10294000660C4B015C016091DE037091DF038091A6
:10295000E0039091E1030E94512C20E030E048EC2C
:1029600052E40E946F2E6B017C010E94F40C20E067
:1029700030E048EC52E40E946F2EA70196010E94BD
:102980006F2E21E03EED42E45EE30E94702F6B016A
:102990007C0120E030E048EC52E4C301B2010E9427
:1029A0006F2EAB01BC0122E0CE0101960E94B9124C
:1029B000BE016F5F7F4F8AE294E00E946A10CE01F1
:1029C00001960E94B5106BE072E08AE294E00E94EA
:1029D00043116AE274E080E394E00E94D2116AEE4F
:1029E00071E0CE0101960E94F2116AE274E0CE011C
:1029F00001960E943011BC018AE294E00E94D2113B
:102A0000CE0101960E94B5106FE172E082E494E07D
:102A10000E944D1121E0B501A401CE0101960E9452
:102A2000B912CE0101960E941111CE0101960E94A9
:102A3000B51068E671E082E494E00E944311A701BA
:102A4000960160E070E080E89FE30E94022E20E0A3
:102A50003AE24DE257E40E94B02CAB01BC0121E008
:102A6000CE0101960E94B912BE016F5F7F4FCE0169
:102A700007960E94E91164EA71E0CE0107960E9470
:102A80001A110E941111CE0107960E94B510CE01B5
:102A900001960E94B5106AE274E0CE0101960E9490
:102AA000E91166EC71E0CE0101960E941A1162E410
:102AB00074E00E943011BC0182E494E00E94D211C3
:102AC000CE0101960E94B51065E070E080E090E0D4
:102AD0000E9425042C960FB6F894DEBF0FBECDBF22
:102AE000DF91CF91FF90EF90DF90CF90BF90AF90AC
:102AF0009F908F907F906F905F904F9008952F924E
:102B00003F924F925F926F927F928F929F92AF927D
:102B1000BF92CF92DF92EF92FF920F931F93CF93CA
:102B2000DF93CDB7DEB7CD54D1090FB6F894DEBF31
:102B30000FBECDBF8C016BE571E082E494E00E9492
:102B40009C11C8010596059740F00C3E2FEF120727
:102B500024F01093A6020093A5020D3F4FEF140737
:102B600009F4C1C60CF0B1C1063F8FEF180709F494
:102B7000BBC10CF0F4C0043FAFEF1A0784F4013F6F
:102B8000BFEF1B070CF0B0C1083E1F4F09F448C748
:102B900066EA72E082E494E00E944D11A5C1043F10
:102BA000FFEF1F0709F434C2053F1F4F89F760E0AC
:102BB00080E10E94B4038091AE02811126C58AE0B3
:102BC00090E0A0E0B0E02E968CAF9DAFAEAFBFAF6F
:102BD0002E9765E372E082E494E00E944D11312C5F
:102BE000212C28961FAE289729961FAE2997C12C15
:102BF000D12C760102E310E0812C912C540180E16C
:102C00000E94E503092E000CAA0BBB0B880E991E2F
:102C1000AA1EBB1E65E070E080E090E00E942504E3
:102C20000150110961F74090FA035090FB03609046
:102C3000FC037090FD03C501B4010E94512C20E0FB
:102C400030E040EA50E40E94B02C20E030E040E860
:102C50005AE30E94B02C20E030E048E452E40E94A5
:102C60006F2EA30192010E94022E20E030E040E787
:102C700051E40E94B02C4B015C01A30192016AE96E
:102C800079E989E390E40E94022E9B01AC01C50121
:102C9000B4010E946F2E20E030E0A9010E94032EB3
:102CA00020E030E040E251E40E94B02C5B018C0156
:102CB000232D322D28964FAD289729965FAD299761
:102CC0000E946B2F181644F43A2C2B2C28960FAF29
:102CD000289729961FAF29979FEFC91AD90AE90AA1
:102CE000F90A2E968CAD9DADAEADBFAD2E978C156D
:102CF0009D05AE05BF050CF07DCF6EE170E080E074
:102D000090E00E94250422E0432D522D28966FADBD
:102D1000289729967FAD2997CE0180960E94B912F7
:102D200069E971E0CE0101960E94F211BE01605E78
:102D30007F4FCE0101960E94301162E474E00E9440
:102D40003011BC0182E494E00E94D211CE010196C0
:102D50000E94B510CE0180960E94B510C5C00B3FF1
:102D60004FEF14070CF0A5C0093F5FEF15070CF0FB
:102D7000BBC0073F8FEF180709F44CC4083F1F4F33
:102D800009F006CF0E9434054B015C0186E794E010
:102D90000E94A20764E670E080E090E00E942504B3
:102DA0000E94B80764E670E080E090E00E9425048D
:102DB00028961FAE2897D12CC12C312C212C2A9675
:102DC0001FAE1EAE2A976CED462E65E0562E612C86
:102DD000712CFE01B0962796FFAFEEAF27970E94A9
:102DE0003405681979098A099B09683B7B4081058C
:102DF000910508F0EBC486E794E00E943707892B21
:102E000009F450C040927A0450927B0460927C0492
:102E100070927D040E94700797FD44C08234910532
:102E2000C9F78E010F5F1F4F78010E94700797FF4F
:102E3000C1C489818D34B1F5C8014D9630E020E0E0
:102E4000D8014D918D01240F311DA817B907C1F785
:102E50002E5B3F4F8E8D90E0982F88274F8D840FEB
:102E6000911D28173907F1F48C8190E0982F88275D
:102E70002D81FC01E20FF11D2A96FFAFEEAF2A97DC
:102E80002E80312C322C22248F81280E311CC884B4
:102E9000D12CDC2CCC248985C80ED11CF1E02896DD
:102EA000FFAF289762E370E080E090E00E94250485
:102EB00096CF0B3FAFEF1A0709F406C50C3F1F4F23
:102EC00009F066CE1092AE020FC00530110509F46C
:102ED0009DC50CF05EC00130110509F410C5C4F5A4
:102EE0000F3F1F4F0CF454CE80914604909147043D
:102EF000892B71F062E474E0CE0101960E94E91121
:102F0000CE0101960E944F12CE0101960E94B5108B
:102F100064E670E080E090E00E942504C35BDF4F30
:102F20000FB6F894DEBF0FBECDBFDF91CF911F91DA
:102F30000F91FF90EF90DF90CF90BF90AF909F9058
:102F40008F907F906F905F904F903F902F9008955B
:102F50000330110509F4DEC40CF4D4C481E080937D
:102F600000010E94DB048C016BE872E082E494E0D3
:102F70000E944D1160E074E0601B710BCE01019660
:102F80000E94A611CE0101960E941111CE01019658
:102F9000E3CE0C30110581F02CF40A3011050CF44D
:102FA000A3CFF6CD0D31110539F00138110521F00F
:102FB0000331110509F0ECCD80910101882309F45A
:102FC00093CF0D31110509F02FC568EE73E080E055
:102FD00090E00E9425040E94851462E474E0CE0112
:102FE00001960E94E911CE0101960E944F12CE0176
:102FF00001960E94B51068E572E080E090E00E94C2
:1030000025046BE571E082E494E00E949C116CCF92
:1030100060E08FE00E94B403E3ECF3E0E491E8A306
:10302000EFEAF3E0E491F0E0EE0FFF1FE457FC4F0E
:10303000859194919AA389A31BA61DA61CA6CE01D7
:10304000809698878F831D821E82198289E08A83E9
:1030500081E08B838C831C8A1B8A1AA619A618A66A
:103060001FA21EA21DA21CA21BA201E0BE01625D46
:103070007F4F8F8198850E94F20E882309F45BC0F0
:1030800067E0CE018E960E9440059DA98913EECF80
:10309000898181111DC08F8198850E94FD05BE0127
:1030A000625D7F4F8F8198850E94DE0540E064EB72
:1030B0008F8198850E94AA058F8198850E94570567
:1030C000182F8F8198850E94FD05111101C0098379
:1030D0001A818EA5803109F4C8C4BE01625D7F4F9C
:1030E000CE0101960E949506811790F48A818A8309
:1030F0008D818F5F8D838EA5883231F0B0F4803161
:1031000019F0823209F0B2CF8E818F5F8E83AECFFD
:103110008EA5803111F48CE0EACFBE01625D7F4F55
:10312000CE0101960E949506E2CF8B3369F382347B
:1031300009F09CCFE9CF8F8198850E94FD0540E082
:103140006CEC8F8198850E94AA05498164E48F8187
:1031500098850E94AA058B81882379F1EA81E9503C
:103160003EEEC32E32E0D32EE33038F4F0E0EE0F23
:10317000FF1FEC5EFE4FC080D1808C81882309F454
:1031800061C0898181115EC00E9434054B015C01E0
:103190000D2C000CEE08FF088F8198850E945705C2
:1031A000813059F00E9434056C197D098E099F0900
:1031B000681579058A059B0578F38CE08A83F12CE4
:1031C000E12C0FE58FE7D82E9FE1C92E2FE3B22E19
:1031D0008D818E151F0409F00CF499C04E2DBE018F
:1031E000695C7F4FCE0101960E94720F1A811D30DB
:1031F00080F11CE08FA9803181F1BE01695C7F4FB5
:10320000CE0101960E949506811709F478C0AE019F
:10321000425D5F4FBE01695C7F4FCE0101960E9407
:103220003506882309F46BC08FA9803109F467C083
:103230001B3009F468C01C3091F01A3009F065C0E9
:10324000BAAA0EC0B601DD0C880B990B0E942504AA
:10325000B4CF193078F619E0CDCF8CE0D5CFDAAA0B
:103260008F8198850E94FD05BE01695C7F4F8F812B
:1032700098850E94DE0540E06EE48F8198850E946B
:10328000AA0540E068A98F8198850E94AA0540E0C0
:1032900069A98F8198850E94AA058FA9803131F094
:1032A00040E06AA98F8198850E94AA058F81988540
:1032B0000E94FD05BE01695C7F4F8F8198850E9449
:1032C000DE05498168E48F8198850E94AA0564E142
:1032D00070E080E090E00E9425048981882331F02D
:1032E0006AE070E080E090E00E9425048F8198857C
:1032F0000E94FD058A81811708F4812F8A83FFEFE0
:10330000EF1AFF0A65CF0AABABCFCAAAA9CFEE80EE
:10331000F12C62E272E0E114F10409F43BCC6BE5BC
:1033200071E082E494E00E949C11670125E0E216BE
:10333000F1041CF014E0C12ED12CBEEFAB2EB3E093
:10334000BB2E10E000E0402FBE01695C7F4FCE0134
:1033500001960E94720F811139C020E030E04EEFDB
:1033600052ECF50161917191819191915F010E94FF
:10337000032E2B013C010F5F1F4F20E030E04CEF8C
:1033800052EC0E944A2C87FF6DC0B801CE01C7964F
:103390000E94A6116EE671E0CE018E960E94F21197
:1033A000BE01695C7F4FCE018E960E94301160E7AE
:1033B00071E00E941A110E941111CE018E960E9496
:1033C000B510CE01C7960E94B51096C0AE01425D01
:1033D0005F4FBE01695C7F4FCE0101960E943506AA
:1033E000882309F4BACF6FA570E0762F6627770F90
:1033F000770F770F2EA548E0249F90011124262BEC
:10340000372B8FA98031D1F46DA970E08CA9DB0135
:10341000A81BB109CD019695982F88279795879578
:103420000E941E31CB014097B901F3E0660F771F70
:10343000FA95E1F760789C01260F371F2138B4EE2A
:103440003B070CF48ACFB901330F880B990B0E940C
:10345000512C20E030E040E05CE30E94B02C9B0166
:10346000AC017FCF22E0B301A201CE01F3E0EF1661
:10347000F10409F474C0CF960E94B912B801CE01CC
:10348000C7960E94A6116EE671E0CE018E960E944C
:10349000F211BE01695C7F4FCE018E960E94301101
:1034A00064E871E00E941A11BE01615C7F4F0E94C6
:1034B0003011BC018AE294E00E94D211CE018E96B6
:1034C0000E94B510CE01C7960E94B510CE01CF96CE
:1034D0000E94B5106AE274E0CE018E960E94E91156
:1034E00066EC71E0CE018E960E941A110E941111B5
:1034F000CE018E960E94B5100C151D050CF423CF3D
:10350000A0904204B0904304A114B10441F0009192
:10351000460410914704650101151105D1F5F3E04A
:10352000EF16F104A9F46CE771E0CE018E960E94CB
:10353000F21162E474E0CE018E960E943011BC015B
:1035400082E494E00E94D211CE018E960E94B510C2
:1035500066E871E082E494E00E944311C5CC8E9647
:103560000E94B912BE01625D7F4FCE01C7960E94D4
:10357000E91166EC71E0CE01C7960E941A110E9413
:103580001111CE01C7960E94B510CE018E961BCFA9
:10359000640146012FEF821A920AD6018C91082EFF
:1035A000000C990B0E94192C892B91F701501109DD
:1035B0000A0D1B1DF8018081082E000C990B0E943A
:1035C000192C892B31F00C151D0518F0015011092B
:1035D000F1CFA8014F5F5F4F4C195D09509347042D
:1035E00040934604AC14BD0420F4B601C5010E940A
:1035F0006E34E0914204F09143048091460490912E
:103600004704E80FF91F10828ACF83E090E0A0E022
:10361000B0E0D9CA68EC70E080E090E00E94250438
:103620000E94080B64E670E080E090E00E942504B0
:1036300062E370E080E090E00E94250449E050E001
:103640006AE171E086E794E00E94130262E370E0B1
:1036500080E090E00E94250403E010E086E794E01B
:103660000E943707892B61F149E050E06AE171E07F
:1036700086E794E00E94130265E070E080E090E04D
:103680000E942504F12CE12C86E794E00E94370784
:1036900092E0E916F104A4F486E794E00E9437076B
:1036A000892B39F086E794E00E944F07AFEFEA1AC2
:1036B000FA0A65E070E080E090E00E942504E4CF23
:1036C00062E370E080E090E00E942504015011095F
:1036D00029F68AE090E00E940E0B6B017C0120E04D
:1036E00030E0A9010E944A2C181634F08AE090E0DC
:1036F0000E940E0B6B017C010BE010E020E030E03B
:1037000042ED53E4C701B6010E944A2C181684F01A
:103710000150110969F068EC70E080E090E00E94CF
:10372000250483E090E00E940E0B6B017C01E6CF44
:1037300020E030E0A901C701B6010E944A2C69E4EB
:1037400072E018160CF026CA20E030E048EC52E493
:10375000C701B6010E944A2C21E087FF20E0B70193
:10376000A601CE0101960E94B912BE016F5F7F4F84
:1037700082E494E00E946A10CE0101960E94B51086
:103780006DE971E0CE0101960E94F21162E474E0ED
:10379000CE0101960E94301162EA71E00E941A1176
:1037A000BC0182E494E00E94D211CE0101960E94F5
:1037B000B5109ACBD7018D937D012796EEADFFAD65
:1037C0002797AE17BF0709F030CB33CB0E943405E3
:1037D000681979098A099B09683B7B408105910535
:1037E000A8F428964FAD2897442309F466C062E3F5
:1037F00070E080E090E00E94250486E794E00E945B
:10380000A20762E370E080E090E06AC028965FADB6
:103810002897552309F451C067E672E082E494E0EA
:103820000E944D11B601CE0180960E94A611B101F1
:10383000CE018E960E94A6112A966EAD7FAD2A9774
:10384000CE01C7960E94A61162E474E0CE01CF9625
:103850000E94E911BE01695C7F4FCE01CF960E94A4
:10386000301166EC71E00E941A11BE01625D7F4F5B
:103870000E94301166EC71E00E941A11BE01605E78
:103880007F4F0E94301166EA71E00E941A11BC015C
:1038900082E494E00E94D211CE01CF960E94B5102E
:1038A000CE01C7960E94B510CE018E960E94B5102B
:1038B000CE0180960E94B5109ACF68E572E082E44E
:1038C00094E00E944D1193CF8091AE02882321F0A5
:1038D00082E494E00E94400268EC70E080E090E0B6
:1038E0000E94250401CB81E08093AE028091A50265
:1038F0009091A6029093A9028093A802F5CA0E9413
:10390000EF12F2CA80910101882309F4EDCA0E94E6
:103910008514EACA8BE0E82EF12C10E000E099242F
:10392000939493E2892E909205038092270310923C
:1039300006031092280362E083E20E94B10910920C
:10394000B8028093B70286EC93E00E948F0AD82ECB
:10395000C12C86EC93E00E948F0A5C01AC28BD2844
:103960000E94CA08B50190E080E00E944F2C2AE92D
:1039700039E949E95FE30E946F2E0E94E82E06179D
:10398000170708F48B0162E370E080E090E00E948A
:10399000250481E0E81AF10831F667E772E082E475
:1039A00094E00E944D1119A218A21BA21AA21DA2F6
:1039B0001CA24AE0BE016F5F7F4FC8010E947828B9
:1039C000BE016F5F7F4FCE0180960E949C116CEA12
:1039D00071E0CE0101960E94F211BE01605E7F4F40
:1039E000CE0101960E94301162E474E00E94301111
:1039F000BC0182E494E00E94D211CE0101960E94A3
:103A0000B510CE0180960E94B510FBCE6BE972E036
:103A100082E494E00E944D110E94DB04BC01AECA16
:103A2000F0E0E0E0099560CA0E94EF1262E474E001
:103A3000CE0101960E94E911CE0101960E944F121B
:103A4000CE0101960E94B51062E370E080E090E044
:103A50000E9425046BE571E082E494E00E949C11D1
:103A60000331110509F440CAB0CA1D3008F03ECB3D
:103A700052CB1F920F920FB60F9211242F933F93A8
:103A80004F935F936F937F938F939F93AF93BF9366
:103A9000EF93FF9389E293E00E94AA02FF91EF91D6
:103AA000BF91AF919F918F917F916F915F914F9156
:103AB0003F912F910F900FBE0F901F9018951F925E
:103AC0000F920FB60F9211242F938F939F93EF9322
:103AD000FF93E0913903F0913A038081E0913F0335
:103AE000F091400382FD1BC09081809142038F5F63
:103AF0008F7320914303821741F0E0914203F0E07D
:103B0000E75DFC4F958F80934203FF91EF919F916A
:103B10008F912F910F900FBE0F901F90189580815D
:103B2000F4CF1F920F920FB60F9211242F933F9351
:103B30008F939F93AF93BF9380919B0290919C0230
:103B4000A0919D02B0919E0230919A0223E0230F32
:103B50002D3758F50196A11DB11D20939A0280932F
:103B60009B0290939C02A0939D02B0939E02809131
:103B70009F029091A002A091A102B091A202019691
:103B8000A11DB11D80939F029093A002A093A1025A
:103B9000B093A202BF91AF919F918F913F912F91CE
:103BA0000F900FBE0F901F90189526E8230F0296D6
:103BB000A11DB11DD2CF1F920F920FB60F921124EB
:103BC0002F933F934F935F936F937F938F939F9325
:103BD000AF93BF93EF93FF93E091B502F091B602DC
:103BE000309749F0A685B7858585968D91FF14C0DD
:103BF0009C918923A1F4FF91EF91BF91AF919F9187
:103C00008F917F916F915F914F913F912F910F9085
:103C10000FBE0F901F9018959C91892361F7A3897F
:103C2000B4899C918589809589238C93868997890D
:103C30000197F1F7608D718DA685B785558538E0C0
:103C400020E0CB010197F1F7822F90E095958795C1
:103C5000282F4C91452309F02068315091F7868D2B
:103C600081FD20958091B40290E001968F73992791
:103C70003091B302381799F0A091B402B0E0A65A7F
:103C8000BD4F2C938093B402828D938D0197F1F7F1
:103C9000A389B4898C919589892B8C93ACCF868D1F
:103CA0008160868FF1CF1F920F920FB60F92112471
:103CB0002F933F934F935F936F937F938F939F9334
:103CC000AF93BF93EF93FF938091B900887F8036C5
:103CD00009F44AC0F0F5883209F4A7C018F580311C
:103CE00009F49BC0B8F4882309F4F9C0883009F4BA
:103CF00094C0FF91EF91BF91AF919F918F917F9170
:103D00006F915F914F913F912F910F900FBE0F9048
:103D10001F901895883109F488C0803251F780933C
:103D2000FD0214C0803409F49DC040F48033B9F31F
:103D30008833F9F68093FD0285ECB0C0803509F434
:103D400085C0883509F496C0883499F60E940C1015
:103D5000D0CF883909F48CC038F5883729F050F471
:103D6000883611F0803729F683E08093FF021092A5
:103D7000590257C0883809F47BC0803919F080385F
:103D800009F0B7CF80915902803208F071C0E091FC
:103D9000590281E08E0F809359028091BB00F0E0C0
:103DA000E75CFD4F80833DC0803B39F0E0F4803A12
:103DB00009F479C0883A09F09CCF84E08093FF022F
:103DC0001092380210923702E091B102F091B202E3
:103DD00009958091370281110FC081E080933702ED
:103DE0001092170209C0803C09F4A6CF883C09F460
:103DF000A3CF883B09F07DCFE091380281E08E0FA0
:103E000080933802F0E0E95EFD4F80818093BB0033
:103E1000909138028091370229C08091DA02809314
:103E2000BB0085EC8093BC0064CF9091FC02809134
:103E3000FB02981758F5E091FC0281E08E0F809309
:103E4000FC02F0E0E552FD4F8081E9CFE091FC02F9
:103E500081E08E0F8093FC028091BB00F0E0E55280
:103E6000FD4F80839091FC028091FB029817C8F26D
:103E700085E8D8CFE091FC0281E08E0F8093FC02B0
:103E80008091BB00F0E0E552FD4F80838091FE02FF
:103E900081115CCF81E08093D90284EA8093BC00D9
:103EA0001092FF0226CF85EC8093BC001092FF0297
:103EB00080915902803230F4E0915902F0E0E75CE1
:103EC000FD4F10826091590270E0E091AF02F091D5
:103ED000B00289E392E00995109259020ACF10923C
:103EE000FD0234CF10922C0310922B0388EE93E046
:103EF000A0E0B0E080932D0390932E03A0932F03B6
:103F0000B093300327E231E030932A032093290352
:103F100025EC30E0309336032093350324EC30E079
:103F2000309338032093370320EC30E030933A038A
:103F30002093390321EC30E030933C0320933B0382
:103F400022EC30E030933E0320933D0326EC30E03A
:103F50003093400320933F03109242031092430397
:103F600010924403109245031092C9031092C803A3
:103F70008093CA039093CB03A093CC03B093CD035B
:103F800029E331E03093C7032093C6031092A204C3
:103F9000109279041092780480937A0490937B04B1
:103FA000A0937C04B0937D048BE491E0909377041C
:103FB0008093760410928D0410928C0410928F04DA
:103FC00010928E0410929104109290041092930417
:103FD00010929204609194046E7F6D7F60939404BC
:103FE0006695617081E0682789E00E94860361E040
:103FF00089E00E94B403EDEBF3E0E491E0938604E2
:10400000E9EAF3E0E491F0E0EE0FFF1FEA56FC4F1F
:1040100085919491909388048093870460E08AE06E
:104020000E94B4038091940481FD04C061E08AE0A1
:104030000E9486038AE080938204EEEBF3E0E49131
:10404000E0938304EAEAF3E0E491F0E0EE0FFF1F6F
:10405000E457FC4F85919491909385048093840458
:104060008FEF809351048093520480935304809384
:1040700054046BE571E082E494E00E94F2116BE578
:1040800071E08CE394E00E94F2116BE571E086E34D
:1040900094E00E94F2116BE571E080E394E00E94ED
:1040A000F2116BE571E08AE294E00E94F2116FEA8E
:1040B00071E084E294E00E94F21166EB71E08EE11F
:1040C00094E00E94F21186E190E09093D3038093F4
:1040D000D2038CE79CE8A1E0B0E08093DE039093EC
:1040E000DF03A093E003B093E10381EA97E6A3E343
:1040F000BDEB8093E2039093E303A093E403B093BA
:10410000E50386E696E6A6EABFE38093E60390938E
:10411000E703A093E803B093E90381E08093F203FF
:1041200029E130E03093F4032093F3038093F50307
:1041300080E090E4ACE1B5E48093F6039093F7035C
:10414000A093F803B093F9031092FA031092FB03C3
:104150001092FC031092FD03EEEFF3E080E1DF012B
:104160001D928A95E9F710920E0410920F04109296
:104170001004109211041092120410921304109261
:104180001404109215041092160410921704109241
:1041900018041092190410921A0410921B04109221
:1041A0001C0410921D040895CF93DF93CDB7DEB7A2
:1041B0002C970FB6F894DEBF0FBECDBF789484B5B0
:1041C000826084BD84B5816084BD85B5826085BD13
:1041D00085B5816085BD80916E00816080936E00A1
:1041E0001092810080918100826080938100809193
:1041F0008100816080938100809180008160809344
:1042000080008091B10084608093B1008091B00003
:1042100081608093B00080917A00846080937A00FE
:1042200080917A00826080937A0080917A00816028
:1042300080937A0080917A00806880937A0010924F
:10424000C10061E08EE00E94B403E0913903F09177
:104250003A0382E08083E0913503F09136031082C7
:10426000E0913703F09138038FEC80831092410383
:10427000E0913D03F0913E0386E08083E0913B03B3
:10428000F0913C03808180618083E0913B03F09159
:104290003C03808188608083E0913B03F0913C0384
:1042A000808180688083E0913B03F0913C038081B2
:1042B0008F7D808360E08EE00E9486030E949208DA
:1042C00081E08093050383E2809327031092060325
:1042D0001092280360E186EC93E00E94D60A0E94C7
:1042E000CA088FE39CE90197F1F700C0000068EC71
:1042F00070E080E090E00E94250484E690E09093D6
:104300000301809302010E94712D8093A30285E630
:1043100090E00E94712D8093A4020091A30210915D
:10432000A402B801012E000C880B990B0E94512C9D
:104330009B01AC010E94C02F811106C00B501109D6
:104340000C30110508F4B4C084E690E00E94DF0F41
:1043500068EC70E080E090E00E9425046AEE72E074
:1043600082E494E00E944D1162E474E0CE01019673
:104370000E94E911CE0101960E944F12CE010196D2
:104380000E94B5100E94920864E670E080E090E020
:104390000E94250486E780934804809151048F3F52
:1043A00011F40E949208809151048F3F01F5809191
:1043B000480491E09093050380932703109206032D
:1043C0001092280360ED86EC93E00E94D60A0E94CA
:1043D000CA0861E0809148040E94B1091092B802B5
:1043E0008093B70286EC93E00E948F0AF82EF8E5DE
:1043F000FF1609F488C06EED72E082E494E00E943A
:104400004D111092010162E474E0CE0101960E9408
:10441000E911CE0101960E944F12CE0101960E9431
:10442000B51098EE892E93E0992EA12CB12C712C09
:10443000612C2AE2E22EF12C80E0C82E80E0D82EFA
:104440006BE571E0CE0107960E94F21110E089E25F
:1044500093E00E948A02181619060CF0C5C01111CB
:10446000C3C089E293E00E9468028A3009F00EC15D
:104470001091A702112309F41EC180913A04909172
:104480003B04892B09F410C16FEB71E0CE0101965A
:104490000E94F211BE01695F7F4FCE0101960E941A
:1044A00030110E944002CE0101960E94B510FCC05E
:1044B00032EDC32E33E0D32E04E610E0C8010E9493
:1044C000712DF60181936F010F5F1F4F003B1105A6
:1044D000A9F78091D2039091D30390930501809323
:1044E000040164ED73E0CE0101960E94F211BE0159
:1044F0006F5F7F4F84E294E00E946A10CE010196C4
:104500000E94B51025CF88E80E94AE0F9093560404
:10451000809355048AE80E94AE0F909358048093CC
:1045200057048CE80E94AE0F90935A04809359046C
:104530008EE80E94AE0F90935C0480935B0480E948
:104540000E94AE0F90935E0480935D0482E90E9406
:10455000AE0F9093600480935F0484E90E94AE0FD5
:10456000909362048093610486E90E94AE0F909359
:1045700064048093630488E90E94AE0F90936604FC
:10458000809365048AE90E94AE0F9093680480933B
:1045900067048CE90E94AE0F90936A0480936904CB
:1045A0008EE90E94AE0F90936C0480936B0480910F
:1045B00051048F3F09F035CF8091480491E09093EA
:1045C000050380932703109206031092280364EFDB
:1045D00086EC93E00E94D60A6FE386EC93E00E949B
:1045E000D60A0E94CA081DCF8B859C85892B51F065
:1045F00089E293E00E94190364E170E080E090E0BA
:104600000E942504BE01695F7F4F86E394E00E940B
:104610006A10CE0107960E94B5106BE571E082E446
:1046200094E00E949C1180913A0490913B04813067
:10463000910509F0C8C066E374E0CE0101960E94BE
:10464000E9118D819E81892B99F0E981FA8130975A
:1046500079F08081823409F44DC07CF58A3209F406
:10466000AFC0813409F43FC061ED71E08332E9F1FC
:10467000BE016F5F7F4F86E394E00E94D2116AE033
:1046800070E080E090E00E94250440C08D3009F485
:10469000EFCE89831A8241E050E0BE016F5F7F4F09
:1046A000CE0107960E94E5106AE070E080E090E09D
:1046B0000E942504CCCE11E0F7CF8136A1F074F42E
:1046C0008334B1F66EEC71E086E394E00E949C11B5
:1046D00021E02093AE028DEF9FEF16C0823651F09D
:1046E000833681F3C5CF68EC71E086E394E00E94E5
:1046F0009C110CC06BEC71E086E394E00E949C116D
:104700001092AE028CEF9FEF0E947F15CE010196B2
:104710000E94B51086E394E00E944410CB010E94F1
:104720007F158091AE02882309F43EC00E943405B3
:10473000A50194010E94D12DCA01B9010E944F2CFC
:104740002091AA023091AB024091AC025091AD028F
:104750000E94022E20910A0130910B0140910C0120
:1047600050910D010E946B2F1816F4F40E9434052D
:10477000A50194010E94D12DCA01B9010E944F2CBC
:104780006093AA027093AB028093AC029093AD0247
:104790008091A8029091A9020E947F156AE070E0C2
:1047A00080E090E00E942504C114D10409F448CEB1
:1047B0000E949602882309F443CE0E9400003CCE5A
:1047C00064ED71E092CF049768F567ED71E0CE017A
:1047D00001960E94F211BE016F5F7F4F86E394E065
:1047E0000E944F10182FCE0101960E94B510112380
:1047F000C9F080913A0490913B04029788F0E091CF
:104800003604F0913704309759F0818180330CF4ED
:10481000845EF701E81BF10987FDF395CF017FCF97
:1048200080E0F6CF66E374E08CE394E00E94D2115E
:1048300000913C0410913D040115110571F0F8013F
:1048400081918F01882349F0082E000C990B0E945A
:104850006634F80131978083F2CF61E773E0CE01CF
:1048600001960E947211BE016F5F7F4F8CE394E04E
:104870000E944F10182FCE0101960E94B5101123EF
:1048800019F0F30109954DCF69E673E0CE01019669
:104890000E947211BE016F5F7F4F8CE394E00E9413
:1048A0004F10182FCE0101960E94B510112399F1D7
:1048B00069ED71E0CE0101960E94F2116EE174E0A3
:1048C000CE0101960E943011BC0182E494E00E9466
:1048D000D211CE0101960E94B51063EE71E0CE01B7
:1048E00001960E94F21162E474E0CE0101960E94EA
:1048F0003011BC01CE0107960E94E911CE01079646
:104900000E944F12CE0107960E94B510CE0101966B
:104910000E94B51006CF62E673E0CE0101960E94B8
:104920007211BE016F5F7F4F8CE394E00E944F10C5
:10493000182FCE0101960E94B510112359F064E59D
:1049400073E082E494E00E944D1184E294E00E94BE
:104950001111C3CF6DE473E0CE0101960E94721174
:10496000BE016F5F7F4F8CE394E00E944F10182FC1
:10497000CE0101960E94B510112311F127E030E01D
:1049800046E050E066E374E0CE0101960E94031217
:10499000BE016F5F7F4F80E394E00E946A10CE01FA
:1049A00001960E94B51080E394E00E944410672BAA
:1049B00019F41092A702B5CEF1E0F093A702B1CEA0
:1049C00066E473E0CE0101960E947211BE016F5F32
:1049D0007F4F8CE394E00E944F10182FCE01019678
:1049E0000E94B510112309F47BC020913A04309144
:1049F0003B042730310508F494CE46E050E066E3EE
:104A000074E0CE0101960E940312BE016F5F7F4FDA
:104A100080E394E00E946A10CE0101960E94B510D6
:104A20008091300490913104009709F455C00E94A0
:104A30001D2860930A0170930B0180930C019093E1
:104A40000D016BE373E082E494E00E944D1140910C
:104A50000A0150910B0160910C0170910D0122E04F
:104A6000CE0101960E94B912BE016F5F7F4FCE0149
:104A700007960E94E91165EE71E0CE0107960E944B
:104A80001A110E941111CE0107960E94B510CE0195
:104A900001960E94B51062E474E0CE0101960E9476
:104AA000E911CE0101960E944F12CE0101960E949B
:104AB000B5100E943405A50194010E94D12DCA01B0
:104AC000B9010E944F2C6093AA027093AB028093AD
:104AD000AC029093AD0225CE60E070E0CB01A9CF8F
:104AE00064E373E0CE0101960E947211BE016F5F14
:104AF0007F4F8CE394E00E944F10182FCE01019657
:104B00000E94B510112309F469C020913A04309134
:104B10003B042730310508F404CE46E050E066E35C
:104B200074E0CE0101960E940312BE016F5F7F4FB9
:104B300080E394E00E946A10CE0101960E94B510B5
:104B40008091300490913104009709F443C00E9491
:104B50001D286093060170930701809308019093CC
:104B6000090169E273E082E494E00E944D114091F2
:104B7000060150910701609108017091090121E03F
:104B8000CE0101960E94B912BE016F5F7F4FCE0128
:104B900007960E94E91165EE71E0CE0107960E942A
:104BA0001A110E941111CE0107960E94B510CE0174
:104BB00001960E94B51062E474E0CE0101960E9455
:104BC000E911CE0101960E944F12CE0101960E947A
:104BD000B510A7CD60E070E0CB01BBCF64E273E01D
:104BE000CE0101960E947211BE016F5F7F4F8CE370
:104BF00094E00E944F10182FCE0101960E94B5102C
:104C0000112341F126E030E044E050E066E374E037
:104C1000CE0101960E940312BE016F5F7F4F80E3B9
:104C200094E00E946A10CE0101960E94B51080E3C4
:104C300094E00E9444107093D3036093D203709366
:104C400005016093040180910201909103010E948B
:104C5000DF0F67CD60E273E0CE0101960E94721112
:104C6000BE016F5F7F4F8CE394E00E944F10182FBE
:104C7000CE0101960E94B510112309F451C0209174
:104C80003A0430913B0443E050E066E374E0CE0127
:104C900001960E940312BE016F5F7F4F80E394E094
:104CA0000E946A10CE0101960E94B51060E374E084
:104CB000CE0101960E94E9111F82188641E050E062
:104CC000BE01695F7F4FCE0101960E94E510811100
:104CD00004C0CE0101960E94A310BE016F5F7F4FFA
:104CE00084E294E00E94D211CE0101960E94B51098
:104CF00000912804109129040115110509F4A3CF8E
:104D0000015011096091240470912504A80184EDDB
:104D100093E00E948C34F801EC52FC4F108293CF48
:104D20006DE173E0CE0101960E947211BE016F5FCA
:104D30007F4F8CE394E00E944F10182FCE01019614
:104D40000E94B510112309F48CC020913A043091CF
:104D50003B042031310508F0E4CC42E050E066E34A
:104D600074E0CE0101960E940312BE016F5F7F4F77
:104D700080E394E00E946A10CE0101960E94B51073
:104D80008091300490913104009799F10E941D2880
:104D900020E030E048EC52E40E94B02C0E94E12E6A
:104DA0006093DE037093DF038093E0039093E1034D
:104DB0008B019C0100591F452140310901341C49D8
:104DC00021053105D0F067EE71E0CE0101960E9419
:104DD000F21160E374E0CE0101960E9430116DEE95
:104DE00071E00E941A11BC0182E494E00E94D21189
:104DF0008DCD60E070E0CB01CBCF0E94512C20E044
:104E000030E048EC52E40E946F2EAB01BC0122E07E
:104E1000CE0101960E94B912BE016F5F7F4F82E4FE
:104E200094E00E946A10CE0101960E94B5106DEFC9
:104E300071E0CE0101960E94F21162E474E0CE01AD
:104E400001960E9430116AE072E00E941A11BC01C2
:104E500082E494E00E94D211CE0101960E94B51026
:104E6000F2CE6FE072E0CE0101960E94F211BE0117
:104E70006F5F7F4F8CE394E00E944F10182FCE019C
:104E800001960E94B510112309F45EC009E110E0FB
:104E9000212C312C210180E10E94E503BC01990FF6
:104EA000880B990B0E94512C9B01AC01C201B101EE
:104EB0000E94032E1B012C016AE070E080E090E06C
:104EC0000E9425040150110931F720E030E040EA4A
:104ED00050E4C201B1010E94B02C20E030EC4FE759
:104EE00054E40E946F2E20E030E048EC51E40E9430
:104EF0006F2E6093FA037093FB038093FC039093EF
:104F0000FD0380910201909103010E94DF0F6AE08E
:104F100073E082E494E00E944D114091FA035091B5
:104F2000FB036091FC037091FD0322E0CE0101962A
:104F30000E94B912BE016F5F7F4FCE0107960E949B
:104F4000E91163E172E029CE66E073E0CE010196DB
:104F50000E947211BE016F5F7F4F8CE394E00E944C
:104F60004F10182FCE0101960E94B510112309F49D
:104F7000D8CB20913A0430913B0443E050E066E303
:104F800074E0CE0101960E940312BE016F5F7F4F55
:104F900080E394E00E946A10CE0101960E94B51051
:104FA00080E394E00E9444107093A6026093A502EF
:104FB000B8CB8EE194E00E94B51084E294E00E94A8
:104FC000B5108AE294E00E94B51080E394E00E945C
:104FD000B51086E394E00E94B5108CE394E00E9443
:104FE000B51082E494E00E94B5108BE491E09093B8
:104FF00077048093760486E794E00C94A207EF92FE
:105000000F931F93CF93DF93E80134E047FD34E122
:10501000042E000C550B57FF03C0519541955109C3
:10502000E32E022F242FAE010E949228CE01DF91A1
:10503000CF911F910F91EF900895662777270C94D9
:10504000F1291F93FC0199278827BC01E89411914D
:105050001032E9F3193010F01E30C8F31B3251F052
:105060001D3249F4689406C00E946328610F711DC7
:10507000811D911D119110531A30B0F33EF490959B
:105080008095709561957F4F8F4F9F4F1F91089529
:10509000FB01DC0105900D920020E1F70895FC0171
:1050A00005900020E9F7809590958E0F9F1F089539
:1050B000BB274A3031F4992322F4BDE290958195C3
:1050C0009F4F0C947928592F482F372F262F660F82
:1050D000771F881F991F660F771F881F991F620F00
:1050E000731F841F951F660F771F881F991F0895D0
:1050F000BB27FB015527AA27880F991FAA1FA417B2
:1051000010F0A41B83955051B9F7A05DAA3308F0A5
:10511000A95DA193009779F7B111B1931192CB01D9
:105120000C943A2CA9E0B0E0E8E9F8E20C94A02D48
:105130006A01F22EB02E102FFBE3AF2EA01608F45A
:105140001BE31F5F012F27E0AE014F5F5F4F0E94FF
:10515000412BBC018981982F9970913009F43FC08F
:105160009BE2E1FC04C09E2D9170E0FC3AC05E2DF4
:105170005071E82FE87083FF46C084E0911101C0B0
:1051800083E0EF2DE81B8F1508F0E0E0D6018E2FAD
:1051900020E2552351F1992329F0D6019C93C601B1
:1051A00001966C0196012D5F3F4FE2FE24C08EE414
:1051B000D6018C9391E411969C93119712968C933F
:1051C000D9018E2F90E281111BC0E20FF32FF11D48
:1051D00010828EEF9FEF2996ECE00C94BC2D9DE29F
:1051E000C6CF90E2C4CF2D9381508111FCCFCE0E5B
:1051F000D11CE0E0D0CF8EE6D6018C9391E6DBCFD8
:105200009D938150E0CF482F447082FF3DC084E0E1
:10521000911101C083E08F1510F4EF2DE81BD6012A
:105220008E2F20E2552309F1992329F0D6019C9372
:10523000C60101966C0196012D5F3F4FE2FE1BC037
:1052400089E4D6018C938EE411968C93119786E4B1
:1052500012968C93D9018E2F90E2882309F4B5CF52
:105260009D938150FACF2D9381508111FCCFCE0EAA
:10527000D11CE0E0D9CF89E6D6018C938EE6119659
:105280008C93119786E6E4CF9B0177FF02C030E054
:1052900020E0A1E0B0E0911102C0B0E0A0E0F9018F
:1052A0003196AE0FBF1F8B2C912CBB2009F461C02F
:1052B0005401EFEFAE1ABE0AAA0DBB1DFA161B066B
:1052C00019F014F04F2D4A1B511188C0E3FC59C04E
:1052D0007601A42FB0E2A1114FC0C40ED11C9923B6
:1052E00009F45BC040E0D6011196F60190836D0190
:1052F000552309F448C0012F060F9A81582F507189
:1053000084FF03C0913309F4015010160CF047C01C
:10531000093008F008E0EEE2FE2E5B01A01AB108A9
:1053200085019194819491082F3F320729F4D60189
:10533000FC92F60131966F016217730794F1021720
:1053400013077CF5DB01A21BB30BAA24A394B12C99
:10535000AC0EBD1EAA0DBB1D11968C9121503109BA
:10536000D601119628153905F4F0F60180836D01F8
:10537000DBCFB12CA12CA0CFF701B1937F01A150BD
:10538000AACF9111B0CFD601942F50E302C05D9304
:1053900091509111FCCFC40ED11C40E0ACCF01E084
:1053A000BACF80E3DBCF6217730731F4963388F40A
:1053B000953311F4552369F0F6018083FD01842FA4
:1053C00090E2811108C0A40FB11D1C9290E080E012
:1053D00002CF81E3F1CF91938150F3CF911183CF2D
:1053E0008ACFB0E0A0E0E7EFF9E20C94A02D5C01D9
:1053F0007B016115710519F0DB018D939C9385018B
:105400000F5F1F4FF501D0818D2F90E00E94192C66
:105410006C01892BB9F5DD32B9F50F5F1F4FD5014E
:105420001196DC91C1E05801F1E0AF1AB10843E0F8
:1054300050E062EF70E0C5010E94222C892B69F5D3
:10544000680182E0C80ED11C45E050E06DEE70E0CE
:10545000C6010E94222C892B21F4680197E0C90E15
:10546000D11CE114F10419F0D701CD92DC9260E077
:1054700070E080E89FEFC111FFC060E070E080E85D
:105480009FE7FAC05801BBCFDB3229F485010E5FDC
:105490001F4FF501D181C0E0C6CF43E050E06AEE76
:1054A00070E0C5010E94222C892BE9F0F80110E080
:1054B00000E020E030E0A9015F01B0ED8B2E8D0E01
:1054C00089E08815C8F19C2E689491F88C2F88701B
:1054D000C2FF16C0811102C00F5F1F4F3196D50168
:1054E000DC91C92DE9CFE114F10429F00E5F1F4FC3
:1054F000F7011183008360E070E080EC9FE7BCC09F
:10550000882311F001501109A5E0B0E00E94872D19
:105510009B01AC01220F331F441F551F280D311D65
:10552000411D511D283999E93907490799E1590762
:10553000A8F2C6609C2ED2CFAEEF8A1206C0C3FD81
:105540003CC09C2E689493F8C9CFDF7DD534A9F573
:1055500080818D3239F4C061DF011296818162E071
:1055600070E006C0DF018B32C1F3119661E070E09C
:1055700080535D01A61AB70A8A30F8F4E0E8CE1627
:10558000ECE0DE065CF4B601660F771F660F771F4E
:10559000C60ED71ECC0CDD1CC80ED11C5D01FFEF62
:1055A000AF1ABF0A8C9180538A30A8F1C4FF03C0A0
:1055B000D194C194D1080C0D1D1DC1FF09C0E11487
:1055C000F10431F081E0A81AB108D701AD92BC9284
:1055D000CA01B9010E944F2CC370C33009F490581E
:1055E0004B015C0120E030E0A9010E944A2C882395
:1055F00009F440C0C1E2D1E017FF05C01195019543
:105600001109C9E0D1E06E01B8E1CB1AD10880E2FE
:10561000E82EF12C0FC0D501B1CFFE0125913591B7
:10562000459154910E191F09C501B4010E94B02C77
:105630004B015C01D501C4010E151F0574F72497B9
:10564000F594E794CC16DD06A9F78A2F880F8B2FE7
:10565000881F8F3F49F020E030E0A901C501B40167
:105660000E944A2C811106C082E290E09093A4042B
:105670008093A304C501B401CDB7DEB7ECE00C9470
:10568000BC2D283008F027E03327DA01990F311DAF
:1056900087FD916000966105710539F432602E5FD7
:1056A0003D9330E32A95E1F708959F3F30F080382D
:1056B0007105610509F03C5F3C5F3D93913008F056
:1056C0008068911DDF93CF931F930F93FF92EF920A
:1056D000192F987F9695E92F96959695E90FFF27B4
:1056E000E158FE4F99273327EE24FF24A701E70155
:1056F00005900894079428F4360FE71EF81E491FFA
:10570000511D660F771F881F991F0694A1F70590FA
:10571000079428F4E70EF81E491F561FC11D770F86
:10572000881F991F661F0694A1F70590079428F417
:10573000F80E491F561FC71FD11D880F991F661FDE
:10574000771F0694A1F70590079420F4490F561F80
:10575000C71FD81F990F661F771F881F0694A9F7C8
:1057600084911095177041F0D695C7955795479538
:10577000F794E7941A95C1F7E5E2F1E06894159083
:10578000159135916591959105907FE27395E1189A
:10579000F10A430B560BC90BD009C0F7E10CF11EFF
:1057A000431F561FC91FD01D7EF4703311F48A9514
:1057B000E6CFE894015030F0080F0AF400270217F2
:1057C00008F4202F2395022F7A3328F079E37D9374
:1057D0002A95E9F710C07D932A9589F60694979546
:1057E0006795379517951794E118F10A430B560BF7
:1057F000C90BD00998F023957E9173957A3308F000
:1058000070E37C932013B8F77E9170617D9330F044
:10581000839571E37D9370E32A95E1F71124EF906E
:10582000FF900F911F91CF91DF91992787FD909560
:10583000089591110C941D2D803219F089508550D6
:10584000C8F70895FB01DC014150504088F08D916C
:1058500081341CF08B350CF4805E659161341CF052
:105860006B350CF4605E861B611171F3990B089522
:10587000881BFCCFDC01FC01672F71917723E1F7D6
:10588000329704C07C916D9370836291AE17BF070D
:10589000C8F308950E948C2C08F481E00895E894E0
:1058A00009C097FB3EF490958095709561957F4F68
:1058B0008F4F9F4F9923A9F0F92F96E9BB27939516
:1058C000F695879577956795B795F111F8CFFAF426
:1058D000BB0F11F460FF1BC06F5F7F4F8F4F9F4F57
:1058E00016C0882311F096E911C0772321F09EE8B5
:1058F000872F762F05C0662371F096E8862F70E01B
:1059000060E02AF09A95660F771F881FDAF7880FF4
:105910009695879597F90895990F0008550FAA0B4A
:10592000E0E8FEEF16161706E807F907C0F01216B2
:105930001306E407F50798F0621B730B840B950BB5
:1059400039F40A2661F0232B242B252B21F408950A
:105950000A2609F4A140A6958FEF811D811D0895A7
:105960000E94C32C0C94372D0E94292D38F00E94E0
:10597000302D20F0952311F00C94202D0C94262D21
:1059800011240C946B2D0E94482D70F3959FC1F348
:10599000950F50E0551F629FF001729FBB27F00DDD
:1059A000B11D639FAA27F00DB11DAA1F649F662732
:1059B000B00DA11D661F829F2227B00DA11D621F81
:1059C000739FB00DA11D621F839FA00D611D221F3B
:1059D000749F3327A00D611D231F849F600D211D1F
:1059E000822F762F6A2F11249F5750409AF0F1F0A2
:1059F00088234AF0EE0FFF1FBB1F661F771F881F0B
:105A000091505040A9F79E3F510580F00C94202DF5
:105A10000C946B2D5F3FE4F3983ED4F38695779515
:105A20006795B795F795E7959F5FC1F7FE2B880FB0
:105A3000911D9695879597F9089599278827089538
:105A400097F99F6780E870E060E008959FEF80EC31
:105A5000089500240A9416161706180609060895D4
:105A600000240A9412161306140605060895092E3A
:105A70000394000C11F4882352F0BB0F40F4BF2BA9
:105A800011F460FF04C06F5F7F4F8F4F9F4F0895E9
:105A900057FD9058440F551F59F05F3F71F04795DF
:105AA000880F97FB991F61F09F3F79F087950895C4
:105AB000121613061406551FF2CF4695F1DF08C0E3
:105AC000161617061806991FF1CF86957105610500
:105AD00008940895E894BB2766277727CB0197F9A8
:105AE0000895F999FECF92BD81BDF89A992780B5A6
:105AF0000895262FF999FECF1FBA92BD81BD20BD12
:105B00000FB6F894FA9AF99A0FBE019608950E947A
:105B1000F32DA59F900DB49F900DA49F800D911D16
:105B200011240895B7FF0C94872D0E94872D821BA6
:105B3000930B08952F923F924F925F926F927F92B4
:105B40008F929F92AF92BF92CF92DF92EF92FF928D
:105B50000F931F93CF93DF93CDB7DEB7CA1BDB0B39
:105B60000FB6F894DEBF0FBECDBF09942A883988DE
:105B700048885F846E847D848C849B84AA84B984E5
:105B8000C884DF80EE80FD800C811B81AA81B981F1
:105B9000CE0FD11D0FB6F894DEBF0FBECDBFED0105
:105BA0000895A1E21A2EAA1BBB1BFD010DC0AA1F5E
:105BB000BB1FEE1FFF1FA217B307E407F50720F076
:105BC000A21BB30BE40BF50B661F771F881F991FF1
:105BD0001A9469F760957095809590959B01AC013A
:105BE000BD01CF010895A29FB001B39FC001A39F43
:105BF000700D811D1124911DB29F700D811D112406
:105C0000911D08955058BB27AA270E941A2E0C9464
:105C1000372D0E94292D38F00E94302D20F039F4C4
:105C20009F3F19F426F40C94262D0EF4E095E7FB23
:105C30000C94202DE92F0E94482D58F3BA176207C3
:105C400073078407950720F079F4A6F50C946A2D64
:105C50000EF4E0950B2EBA2FA02D0B01B901900187
:105C60000C01CA01A0011124FF27591B99F0593FCB
:105C700050F4503E68F11A16F040A22F232F342F13
:105C80004427585FF3CF469537952795A795F04061
:105C90005395C9F77EF41F16BA0B620B730B840B76
:105CA000BAF09150A1F0FF0FBB1F661F771F881F2E
:105CB000C2F70EC0BA0F621F731F841F48F4879586
:105CC00077956795B795F7959E3F08F0B0CF939578
:105CD000880F08F09927EE0F9795879508950E94F1
:105CE000832E0C94372D0E94302D58F00E94292DC0
:105CF00040F029F45F3F29F00C94202D51110C94B1
:105D00006B2D0C94262D0E94482D68F39923B1F336
:105D1000552391F3951B550BBB27AA2762177307D1
:105D2000840738F09F5F5F4F220F331F441FAA1F65
:105D3000A9F335D00E2E3AF0E0E832D09150504021
:105D4000E695001CCAF72BD0FE2F29D0660F771FCF
:105D5000881FBB1F261737074807AB07B0E809F0B5
:105D6000BB0B802DBF01FF2793585F4F3AF09E3F3A
:105D7000510578F00C94202D0C946B2D5F3FE4F3CB
:105D8000983ED4F3869577956795B795F7959F5F7D
:105D9000C9F7880F911D9695879597F90895E1E0C9
:105DA000660F771F881FBB1F621773078407BA0728
:105DB00020F0621B730B840BBA0BEE1F88F7E09583
:105DC00008950E94E82E6894B1110C946B2D0895EB
:105DD0000E94502D88F09F5798F0B92F9927B751FE
:105DE000B0F0E1F0660F771F881F991F1AF0BA957F
:105DF000C9F714C0B13091F00E946A2DB1E0089546
:105E00000C946A2D672F782F8827B85F39F0B93F37
:105E1000CCF3869577956795B395D9F73EF4909531
:105E20008095709561957F4F8F4F9F4F089597FB99
:105E300016F40E945B2F0C941E2FE894F92F96EB1A
:105E4000FF2381F0121613061406440B9395F69562
:105E500087957795679557954040FF23B9F71BC005
:105E600099270895882351F49850D2F7872B762FDD
:105E7000652F542F432F322F20E0B1F31216130653
:105E80001406440B88233AF09A95440F551F661F59
:105E9000771F881FCAF755234AF4440F551F11F482
:105EA00060FF04C06F5F7F4F8F4F9F4F880F9695A5
:105EB000879597F908959095809570956095509580
:105EC0004095309521953F4F4F4F5F4F6F4F7F4F1C
:105ED0008F4F9F4F08950E948C2C08F48FEF0895E8
:105EE000FA01EE0FFF1F309621053105A1F1611572
:105EF000710561F48038BFE39B0749F168949038DD
:105F0000810561F08038BFEF9B0741F099234AF586
:105F1000FF3FE1053105210519F1E8940894E79563
:105F2000D901AA2329F4AB2FBE2FF85FD0F310C0FC
:105F3000FF5F70F4A695E0F7F73950F019F0FF3ADB
:105F400038F49F779F930DD00F9007FC90580895D9
:105F500046F00C94262D60E070E080E89FE3089501
:105F60004FE79F775F934F933F932F930E9470303B
:105F70002F913F914F915F910E94B02C0C94CD2FA7
:105F80000E948C2C880B990B089529F416F00C9420
:105F9000202D0C946A2D0C94262D0E94502DA8F3D0
:105FA0009638A0F707F80F92E8942BE33AEA48EB0B
:105FB0005FE70E94C62C0F920F920F924DB75EB70B
:105FC0000F920E94B830E8E6F0E00E94FF2F4F9158
:105FD0005F91EF91FF91E595EE1FFF1F49F0FE578E
:105FE000E0684427EE0F441FFA95E1F74195550B01
:105FF0000E9432300F9007FE0C9426300895DF93F4
:10600000CF931F930F93FF92EF92DF927B018C014E
:10601000689406C0DA2EEF010E94C32CFE01E894BA
:10602000A5912591359145915591A6F3EF010E94D7
:106030001A2EFE019701A801DA9469F7DF90EF901C
:10604000FF900F911F91CF91DF9108959B01AC01BB
:1060500060E070E080E89FE30C946F2E0C94202D9C
:106060000C94EC300E94502DD8F39923C9F3940F6F
:10607000511DA3F39150504094F059F0882332F011
:10608000660F771F881F91505040C1F79E3F510502
:106090002CF7880F911D9695879597F908955F3F86
:1060A000ACF0983E9CF0BB27869577956795B795A1
:1060B00008F4B1609395C1F7BB0F58F711F460FF76
:1060C000E8CF6F5F7F4F8F4F9F4FE3CF0C946B2DC7
:1060D00016F00C94EC300C94262D68940C94202D22
:1060E0000E94502DA8F39923C1F3AEF3DF93CF9311
:1060F0001F930F93FF92C92FDD2788232AF0219742
:10610000660F771F881FDAF720E030E040E85FEB8A
:106110009FE3883920F0803E38F021968F770E94E7
:10612000032EE0E9F0E004C00E94032EEDEBF0E066
:106130000E94FF2F8B01BE01EC01FB2E6F577109EE
:106140007595771F880B990B0E94512C28E132E737
:1061500041E35FE30E94C32CAF2D9801AE01FF9095
:106160000F911F91CF91DF910E941A2E0C94372D21
:10617000FA01DC01AA0FBB1F9B01AC01BF5728F439
:10618000222733274427507820C0B75190F4AB2FF3
:106190000024469537952795011CA395D2F300203E
:1061A00071F0220F331F441FB395DAF30ED00C9415
:1061B000022E61307105A0E88A07B94630F49B01D0
:1061C000AC016627772788279078309621F02083C6
:1061D00031834283538308959F3F31F0915020F4DF
:1061E000879577956795B795880F911D96958795B3
:1061F00097F90895DB018F939F930E94872DBF919C
:10620000AF91A29F800D911DA39F900DB29F900D05
:1062100011240895AA1BBB1B51E107C0AA1FBB1F75
:10622000A617B70710F0A61BB70B881F991F5A9522
:10623000A9F780959095BC01CD01089597FB072E95
:1062400016F4009407D077FD09D00E940A3107FCAC
:1062500005D03EF4909581959F4F08957095619576
:106260007F4F0895DF93CF931F930F939A9DF02D47
:10627000219FF00D8B9DF00D8A9DE02DF10D039F68
:10628000F00D029FE00DF11D4E9DE00DF11D5E9D94
:10629000F00D4F9DF00D7F936F93BF92AF925F9380
:1062A0004F93D5010E94F32D8B01AC01D7010E94C1
:1062B000F32DEB01E80FF91FD6010E9481312F91D8
:1062C0003F91D6010E94F32DC60FD71FE81FF91F7B
:1062D000AF91BF910E9481312F913F910E94F32D88
:1062E000C60FD71FE81FF91FD6010E94F32DE60F36
:1062F000F71F9801BE01CF010F911F91CF91DF9140
:1063000008950E94F32D460F571FC81FD91F08F488
:1063100031960895689401C0E894F92FF12B12F09A
:106320000C94BE31A0E0B0E0E8E9F1E30C94A02DBC
:10633000092E059422F40E941A32112392F4F0E8F7
:106340000F26FFEFE094F09400951095B094C09460
:10635000D094A194BF0ACF0ADF0AEF0AFF0A0F0BFD
:106360001F0B0E94C93107FC0E941A32CDB7DEB75D
:10637000ECE00C94BC2D689401C0E8948F929F923D
:10638000CF93DF930E94C931DF91CF919F908F907F
:10639000089588249924F401E401B0E49F93AA2786
:1063A0009A158B049C04ED05FE05CF05D007A107C7
:1063B00098F4AD2FDC2FCF2FFE2FE92D982C892EAE
:1063C000982F872F762F652F542F432F322F222778
:1063D000B85031F7BF9127C01B2EBF91BB27220FAA
:1063E000331F441F551F661F771F881F991F881C66
:1063F000991CEE1FFF1FCC1FDD1FAA1FBB1F8A1495
:106400009B04EC05FD05CE05DF05A007B10748F0AC
:106410008A189B08EC09FD09CE09DF09A00BB10B16
:1064200021601A94E1F62EF49401AF01BE01CD0172
:10643000000C0895609570958095909530954095E5
:10644000509521953F4F4F4F5F4F6F4F7F4F8F4F6D
:106450009F4F0895002E083090F0982F872F762FA9
:10646000652F542F432F322F22270850F4CF220FAD
:10647000331F441F551F661F771F881F991F0A95DA
:10648000B2F7002D089597FD1094002E083098F073
:106490000850232F342F452F562F672F782F892F01
:1064A000912DF4CF15949795879577956795579586
:1064B0004795379527950A95AAF71124002D089539
:1064C0002A0D3B1D4C1D5D1D6E1D7F1D801F911FE4
:1064D00008952A193B094C095D096E097F09800B53
:1064E000910B08950024A7FD00942A17300540055C
:1064F000500560057005800590050895EE0FFF1F9B
:106500000590F491E02D09940F931F93CF93DF939F
:106510008230910510F482E090E0E091A704F091C0
:10652000A80430E020E0B0E0A0E0309799F4211515
:10653000310509F44AC0281B390B24303105D8F540
:106540008A819B816115710589F1FB0193838283A7
:10655000FE0111C040815181028113814817590702
:10656000E0F04817590799F4109761F012960C93D0
:10657000129713961C933296CF01DF91CF911F9102
:106580000F9108950093A7041093A804F4CF211548
:10659000310551F04217530738F0A901DB019A0188
:1065A000BD01DF01F801C1CFEF01F9CF9093A8043D
:1065B0008093A704CDCFFE01E20FF31F8193919347
:1065C0002250310939832883D7CF2091A5043091F7
:1065D000A604232B41F42091100130911101309336
:1065E000A6042093A50420910E0130910F012115DE
:1065F000310541F42DB73EB740911201509113017E
:10660000241B350BE091A504F091A604E217F307D3
:10661000A0F42E1B3F0B2817390778F0AC014E5F12
:106620005F4F2417350748F04E0F5F1F5093A604A5
:106630004093A504819391939FCFF0E0E0E09CCF3D
:10664000CF93DF930097E9F0FC0132971382128217
:10665000A091A704B091A804ED0130E020E01097CC
:10666000A1F420813181820F931F2091A5043091E4
:10667000A6042817390709F061C0F093A604E09337
:10668000A504DF91CF910895EA01CE17DF07E8F561
:106690004A815B819E0141155105B1F7E901FB83F8
:1066A000EA8349915991C40FD51FEC17FD0761F496
:1066B000808191810296840F951FE90199838883D7
:1066C000828193819B838A83F0E0E0E012968D9132
:1066D0009C9113970097B9F52D913C911197CD019D
:1066E0000296820F931F2091A5043091A6042817CB
:1066F000390739F6309751F51092A8041092A70483
:10670000B093A604A093A504BCCFD383C2834081D9
:106710005181840F951FC817D90761F44E5F5F4FF1
:1067200088819981480F591F518340838A819B81B9
:10673000938382832115310509F0B0CFF093A8042B
:10674000E093A7049ECFFD01DC01C0CF138212822B
:10675000D7CFB0E0A0E0EFEAF3E30C949C2D8C01DE
:10676000009751F4CB010E9484328C01C801CDB74F
:10677000DEB7E0E10C94B82DFC01E60FF71F9C0199
:1067800022503109E217F30708F49DC0D901CD91D9
:10679000DC911197C617D70798F0C530D10530F3B3
:1067A000CE0104978617970708F3C61BD70B2297CD
:1067B000C193D1936D937C93CF010E942033D6CFA8
:1067C0005B01AC1ABD0A4C018C0E9D1EA091A70462
:1067D000B091A804512C412CF12CE12C109731F5EB
:1067E0008091A5049091A6048815990509F05CC0D4
:1067F0004616570608F058C080910E0190910F017F
:10680000009741F48DB79EB740911201509113014A
:10681000841B950BE817F90708F055C0F093A60400
:10682000E093A504F90171836083A0CF8D919C91C1
:10683000119712966C90129713967C901397A81547
:10684000B90559F56C0142E0C40ED11CCA14DB0431
:1068500020F1AC014A195B09DA011296159780F014
:106860006282738251834083D9016D937C93E114DA
:10687000F10471F0D7011396FC93EE93129776CF43
:1068800022968C0F9D1FF90191838083F301EFCF36
:10689000F093A804E093A70469CF4816590608F4BA
:1068A0002C017D01D3019ACFCB010E9484327C015F
:1068B000009749F0AE01B8010E946E34C8010E94F1
:1068C0002033870153CF10E000E050CF911108959D
:1068D00081568A5108F4805285580895FB01DC01E5
:1068E00002C001900D9241505040D8F70895FB012D
:1068F000DC0101900D920020E1F70895FB01DC011D
:106900004150504030F08D910190801919F40020D1
:10691000B9F7881B990B0895FB01DC0141505040E9
:1069200048F001900D920020C9F701C01D9241501E
:106930005040E0F7089511E0C5EED1E004C0FE013B
:106940000E947E322196C63ED107C9F7F894FFCF48
:106950000101640016000000A0400000F0410000AA
:10696000A90480005E00BC007701FF0186000000E2
:1069700000007900000000CC021302590219038ABA
:106980000268027C0200000000D60AA90A050BDAA0
:1069900006A20A8F0A800A00000000DB0613020527
:1069A0000BDA0637074F07C2060D0A00543D006F89
:1069B000432000483D0025006F4320413D00540026
:1069C0003D4E6F2053656E736F7221005428312C39
:1069D000322C33293D00206F4320445320546865F6
:1069E000726D6F6D657465720055563D00434F3290
:1069F0003D0070706D00206E672F4C004C3D0042D2
:106A00004E4D4C3033004E616E6F42326435007330
:106A1000657269616C3A20002D35002D34002D33EC
:106A2000002D32002D3100440056657273696F6E7F
:106A30003A200023007300534C20503D0050612049
:106A4000697320756E6C696B656C792100536561A3
:106A5000206C6576656C20503D00206850610055C3
:066A6000565A005620000A
:107E0000112484B714BE81FFF0D085E080938100F7
:107E100082E08093C00088E18093C10086E0809377
:107E2000C20080E18093C4008EE0C9D0259A86E02C
:107E300020E33CEF91E0309385002093840096BBD3
:107E4000B09BFECF1D9AA8958150A9F7CC24DD24C4
:107E500088248394B5E0AB2EA1E19A2EF3E0BF2EE7
:107E6000A2D0813461F49FD0082FAFD0023811F036
:107E7000013811F484E001C083E08DD089C08234E0
:107E800011F484E103C0853419F485E0A6D080C0E4
:107E9000853579F488D0E82EFF2485D0082F10E0AE
:107EA000102F00270E291F29000F111F8ED06801E7
:107EB0006FC0863521F484E090D080E0DECF843638
:107EC00009F040C070D06FD0082F6DD080E0C81688
:107ED00080E7D80618F4F601B7BEE895C0E0D1E017
:107EE00062D089930C17E1F7F0E0CF16F0E7DF06D8
:107EF00018F0F601B7BEE89568D007B600FCFDCFD4
:107F0000A601A0E0B1E02C9130E011968C91119780
:107F100090E0982F8827822B932B1296FA010C0160
:107F200087BEE89511244E5F5F4FF1E0A038BF0790
:107F300051F7F601A7BEE89507B600FCFDCF97BE46
:107F4000E89526C08437B1F42ED02DD0F82E2BD052
:107F50003CD0F601EF2C8F010F5F1F4F84911BD097
:107F6000EA94F801C1F70894C11CD11CFA94CF0C13
:107F7000D11C0EC0853739F428D08EE10CD085E9AC
:107F80000AD08FE07ACF813511F488E018D01DD067
:107F900080E101D065CF982F8091C00085FFFCCF94
:107FA0009093C60008958091C00087FFFCCF809118
:107FB000C00084FD01C0A8958091C6000895E0E648
:107FC000F0E098E1908380830895EDDF803219F02E
:107FD00088E0F5DFFFCF84E1DECF1F93182FE3DFCA
:107FE0001150E9F7F2DF1F91089580E0E8DFEE27F6
:047FF000FF270994CA
:027FFE00040479
:00000001FF
